:10000000027537027A4300000000000270BD000054
:10001000000000027AA10000000000022FD20000C0
:10002000000000023B5F000000000002723A000086
:1000300000000000000000000000000000000000C0
:100040005052333032207665722E322E30332E31BC
:10005000353430202847292032352D30312D3130AC
:100060002030323A30312075F00612011D22127014
:100070000C75F00612011D1270132212006E120090
:100080006712006E12006712006E12006712006E97
:1000900012006712006E75F01812011D2212700C0A
:1000A00075F04B12011D12701322754E041233E1CC
:1000B0001233F712700C75F0C812011D1270132262
:1000C000754E051233E11233F712009D75F01E12C2
:1000D000011D12009D22754E071233E11233F712F3
:1000E000008722754E061233E11233F712008D227B
:1000F00012007B12007B221200E31200E31200E3E5
:1001000022C2A1C24A12006E75F01212011DD2A1C4
:10011000C24A2212006E75F01212011D221296259B
:10012000201D07C0F01292BCD0F0D5F0F022700470
:10013000A238B322C0E01478A212013FD0E022C05E
:10014000E0030303540F28F8D0E0C0E0540704F59F
:10015000F0E213D5F0FCD0E0227003D3802830E722
:1001600003C3802223F9C3137004A238801814C07B
:10017000E0030303540F24A2F8D0E0540704F5F081
:10018000E213D5F0FCE992E022C0E024C2F8E212CA
:1001900001594004D0E0C322D0E024D8F582740095
:1001A0003400F583E01201A92220E702C322C2E74E
:1001B000C0E0C2E0700AA238B3D0E030E001B32260
:1001C000B47E03C380F3B40204A22280ECB404041E
:1001D000A22380E5B40604A22480DEB40A04A2149B
:1001E00080D7B40C0AE5684569C36001D380CAB4FE
:1001F0000E05126A4F80C2B41007A24F724EB38030
:10020000B8B41206A24E821580AFB41406A24EB046
:100210001580A6B41604A24F809FB418077400126C
:100220007EB28095B41A077401127EB2808BB41C22
:10023000077402127EB28081B41E087403127EB26B
:100240000201B9B420087404127EB20201B9B422CA
:10025000087405127EB20201B9B424087406127E35
:10026000B20201B9B426087407127EB20201B9D0F5
:10027000E0C3221202AD307005C270126D2F124120
:1002800099E5616013B401051202C68008B4020545
:100290001202ED80007561001292BCE56A54406064
:1002A0000B20A808304705C24712932F22306A1549
:1002B000C26AA2AFC0D0C2AF12970D129625120625
:1002C00087D0D092AF22C238757A1FD263C2AF7581
:1002D000186075190F751AFA1297231212AF12557A
:1002E000A3757303120C7A1296FDC23A22D23875A6
:1002F0007A1FC263C2AF75187075190F751AFA129A
:10030000972312559475730322C2B61278967537E7
:10031000007403125608E51E125608E51F1256080F
:10032000745712560812033AE53712560874FF1232
:1003300056083099FD129659D3227893E612560842
:100340007892E630E402240A540F1256087891E6B7
:10035000C4540375F00AA4F5F0E6540F25F01256C4
:10036000087890E6C4540375F00AA4F5F0E6540F3B
:1003700025F0125608788FE6C4540775F00AA4F5E4
:10038000F0E6540F25F0125608788EE6C45407752F
:10039000F00AA4F5F0E6540F25F01256087892E61C
:1003A00003C454071256082275F032129641129770
:1003B0000D12964112970DD5F0F122D2A3C248D268
:1003C000A2C24BC2A1C24AD2A4C24912700C1203EB
:1003D000A81270131203A812700C1203A812701343
:1003E0001203A812700C1203A81270131203A812A1
:1003F00003A81203A81203A81203A82275F0FFC0D5
:10040000F012067AD0F030E70820E50530E302C3A9
:100410002274C8D5E0FDD5F0E6D32275F0FFC0F018
:1004200012067AD0F030E70820E50530E302C32257
:100430000000000000D5F0E6D322C0F012041B50EB
:100440002912041B502412041B501F12041B501AA3
:100450001203FC50151203FC50101206871203FC05
:1004600050081206871203FC4003D0F022120687C0
:100470001203BB1203FC50F2C2AF7518C07519000D
:10048000751A591297231203BB75F0FA129625D5E7
:10049000F0FA027467AAF012043AE532652FF5F01B
:1004A000E533653045F0600C1205C9852F32853083
:1004B0003312043A12063F12043A12066712043A43
:1004C0001205D68AF022AAF012043AE532652FF519
:1004D000F0E533653045F0600C1205C9852F328593
:1004E000303312043A12062B12043A120667120431
:1004F0003A1205D68AF022E53129501C601AC0E074
:10050000F5F0E9C395F0F928C0E0120518D0E0F83D
:10051000D0E0F9053075310012043AE532652FF567
:10052000F0E533653045F0600C1205C9852F328542
:10053000303312043A1205FB22AAF0E53129501C8F
:10054000601AC0E0F5F0E9C395F0F928C0E01205A3
:100550005CD0E0F8D0E0F9053075310012043AE5DE
:1005600032652FF5F0E533653045F0600C1205C9B2
:10057000852F3285303312043A1205E38AF022C007
:10058000F075F00833C297929000D297D5F0F5D06D
:10059000F022C0F075F008C297D29700A29133D52F
:1005A000F0F5D0F022D292D297D290D291D293226B
:1005B00012057FE53033E52F3312057FC3E5303375
:1005C00012057FE53112057F221205A5C2937453EF
:1005D0001205B0D293221205A5C29374581205B029
:1005E000D293221205A5C29374541205B0E41205E9
:1005F0007F120592F608D9F9D293221205A5C2936B
:1006000074541205B0E412057F120592F208D9F96C
:10061000D293221205A5C29374541205B0E41205B8
:100620007F120592F0A3D9F9D293221205A5C293A5
:1006300074841205B0E612057F08D9F9D29322120C
:1006400005A5C29374841205B0E212057F08D9F99A
:10065000D293221205A5C29374841205B0E012054C
:100660007FA3D9F9D293221205A5C29374831205F0
:10067000B0D29312962512962522C2937457120572
:100680007F120592D29322D290D291D297D292D257
:100690009312970D75F002129625D5F0FAC29212B8
:1006A000970D75F002129625D5F0FAD2927532FFA9
:1006B0007533FF12970D227900752F0175300F7574
:1006C00031009000EE12043A1205C912043A1206E3
:1006D00013852F32853033227900752F0175301044
:1006E0007531009000EE12043A1205C912043A1254
:1006F0000613852F32853033227583007582CF74BF
:1007000010120799227400258274F03583403D74DD
:10071000002582F58274CF3583F5837401F9748CDA
:10072000F8752F00858330858231120539788CE683
:10073000601AB4FF02C322167401F9748CF8752F85
:10074000008583308582311204C6C322D32274000F
:100750002DF58274CF3EF5837401F9748CF8752FF2
:1007600000858330858231120539788CE6FC22744D
:10077000002D74F03E402174002DF58274CF3EF5BB
:1007800083788CECF67401F9748CF8752F008583EE
:10079000308582311204C6C322F5F085832F85820D
:1007A00030753100C0F0C082C08312043A12086272
:1007B000D083D082D0F0A3D5F0E17532FF7533FF3E
:1007C00022F5F0C0F0C082C0838F2F8E30753100CB
:1007D00012043A1205C9D083D082C082C0838583B7
:1007E0002F85823075310012043A120667D083D00B
:1007F0008205820ED0F0D5F0CA7532FF7533FF2224
:10080000758302758200748E120799758303758251
:100810000074F9120799227F027E007583007582A9
:1008200000748E1207C17F037E00758301758200FC
:1008300074F91207C1227F007E0075830275820061
:10084000748E1207C17F017E007583037582007468
:10085000F91207C1221205A5C29374501205B0D235
:1008600093221205A5C29374811205B0D29322126D
:1008700005A5C29374841205B0E812057FD9FAD297
:100880009322F8790012043A12086FEAC0E08582D8
:100890002F85833075310012043A120667D0E0FAD2
:1008A0000583DAE77532FF7533FF221205A5C2937F
:1008B00074541205B0E412057FE4C0E0120592D032
:1008C000F025F0D9F5D29322758302758200800657
:1008D000758300758200E475F08D85832F858230E5
:1008E000753100C082C083C0F0C0E012043A120526
:1008F000C912043A79001208ABD0F025F0D0F0D03C
:1009000083D0820582D5F0D285832F8582307531E0
:1009100000C0E012043A1205C912043A7920120804
:10092000ABD0F025F07532FF7533FF227583037568
:1009300082008006758301758200E475F0F9858375
:100940002F858230753100C082C083C0F0C0E012B4
:10095000043A1205C912043A79001208ABD0F02506
:10096000F0D0F0D083D0820582D5F0D27532FF75F9
:1009700033FF05E022758300758200748E1207999B
:1009800075830175820074F912079922C0E012057F
:10099000A5C29374541205B0E412057F79001205C4
:1009A00092F5F0D0E0C0E0B5F008D9F2D293D0E0F3
:1009B000C322D0E0D322F5F085832F8582307531B4
:1009C00000C082C083C0F012043A1205C912043A72
:1009D00074FF12098CD0F0D083D082400D0582D5EF
:1009E000F0D67532FF7533FFC3227532FF7533FFC2
:1009F000D3227892E603C45407788CF63012257817
:100A000091E6540FC0E0E6C4540375F00AA4D0F098
:100A100025F0FD7892E630E402240A540FFE900D92
:100A200000120A25227F807404F97400F8752F01E2
:100A3000858330858231C0F01204F7D0F07800E26F
:100A40006D700C08E26E700708E2788CF6D322A372
:100A5000A3A3A3DFD2C322C25B1278961209F212BB
:100A600078CDFEAFF07DFF0DBD00051206B7800604
:100A7000BD40031206D8ED30E70122D252C2E6751E
:100A8000F004A424EEF582E5F03400F583788CE0E0
:100A9000F6A308E0F6A308E0F6A308E0F6788C8653
:100AA00083088682788CB6FF0708B6FF03020B33F3
:100AB000C3E58233F582E58333F583E5822400F5CF
:100AC00082E5833411F583788EE6706708E660630B
:100AD000FB7402F9748CF8752F018583308582319F
:100AE000120539A3A3788CE60856B4FF03020B3332
:100AF000788C86F053F07F08E6C39EC5F09F402AAD
:100B00007031E5F06024BD002F2038532037507835
:100B10008CE6A2E720E748C0F01224D2D0F0B5F06E
:100B200000403CD25BD25D020B5F788CE6A2E7927C
:100B300052DB9EBD00028027ED14C0E00303035486
:100B40000F24A2F8D0E0540704FBE4D333DBFD30DC
:100B50005205FBE24B8004F4FBE25BF2020A6712EF
:100B60009308406AB252202C6520624030520D201A
:100B7000375C78BEE2600BD25D020BCE30374F029D
:100B80000BAC78BCE26025C26312747E601EF5F087
:100B9000E5F0543F4400C2AF7518C0751909F51A45
:100BA00012972378BCE278BEF2020BCEC262120C1E
:100BB0007AA25292374011303814E56E5410700EFC
:100BC000120C871254DD8006203803120CA5020A8D
:100BD00067FF305D5978BEE2700C205B34302C51D9
:100BE000205E41020C31BF0003020C0014F27010B1
:100BF00078BCE2603C12747E603778BCE278BEF26A
:100C00001224D2602CF5F078BEE2C5F0B5F00040B9
:100C100020205C10D25CC2AF7518C0751900751A1F
:100C20005D129723E56D540170071200E322120C48
:100C30007AC25C22FF78BF203826303723E2602258
:100C4000BF00221224D2601AF5F078BFE2C5F0B5D9
:100C5000F000400ED273E56D540170031200E322E0
:100C6000E4F2C2732278BFE214F270D7D262120AA1
:100C7000573038EE1200D6C27322C25EC25BC25C2D
:100C8000C25DE478BEF222C238D263C2AF7518608A
:100C900075190F751AE01297231255A37573031275
:100CA00096FDC23A22D238C263C2AF751870751968
:100CB0000F751AE0129723125594757303221205CB
:100CC0007FE53033E52F3312057FC3E53033D2E0C3
:100CD00012057FE53112057F221205A5C2937454D7
:100CE000120CBEE412057F120592F608D9F9D293D0
:100CF000221205A5C2937484120CBEE612057F0869
:100D0000D9F9D2932290FC00752F0475300075310B
:100D100000C082C0837548FA12043A1205C9852FB3
:100D20006085305F7908788C12043A120CD9120F62
:100D300049D083D0827044C082C083789086830873
:100D40008682120DB24024788E8683088682120D28
:100D5000B24018120DC1E582600AE55DB55F0CE591
:100D60005EB56007D083D082020D8D788EE6249A1E
:100D7000F6120F8C1203BBD083D0820530E53070A1
:100D800002052FA3E58245837087120D947532FF0B
:100D90007533FF22788E760008760078907600080A
:100DA0007600087600087600756004755F00120F03
:100DB0006822E5822400E58334804001229000000F
:100DC00022E58275F008A4F582E5F0C58375F00888
:100DD000A42583F583E5F03404F55EE5822400F56F
:100DE00082E5833400F5835002055E85835D22121F
:100DF00003BBD083D08222C082C083120F2270EF47
:100E0000788E8683088682120DB240E3120DC112DD
:100E1000121D788C76007890E518F608E519F6082A
:100E200076000876007408F9748CF8855E2F858347
:100E3000308582311204C67404F97490F8855E2FEF
:100E400085833085823112053975F004788C79906C
:100E5000E667600280990809D5F0F5120F29788EAF
:100E60008683088682A3120DB2788EA68308A68296
:100E700078908683088682120DB2788EE66583703C
:100E80006208E66582705CC05EC05DC082C083128D
:100E90000DC17408F97494F8855E2F8583308582BE
:100EA00031120539789876C00876570876000876AA
:100EB00000D083D082E582241EF582500205831281
:100EC0000DB2C082C083120DC17408F97494F88504
:100ED0005E2F8583308582311204C6D083D082D0C4
:100EE0005DD05E7890A68308A682C060C05F855EF4
:100EF00060855D5F120F68D0E0D0F0B55F09C5F086
:100F0000B560028018C5F0C060C05F85F060F55F15
:100F1000788EE62499F6120F8CD05FD060D083D003
:100F20008222120F29120F492285602F855F3075AA
:100F3000310012043A1205C97908788C12043A1269
:100F40000CD9852F32853033227891E61826182661
:100F5000182618245566700F7891E61866186618DA
:100F60006618661864996622120F6F120F8C227829
:100F700091E6182618261826182455F67891E618B2
:100F800066186618661866186499F62285602F85BB
:100F90005F3075310012043A1205C912043A79081B
:100FA000788C120CF112043A12066712043A1205F8
:100FB000D6852F3285303322120F227030788EE69C
:100FC000C0E008E6C0E0088683088682C3D0E095CA
:100FD00082F582D0E09583F58350104582600CE560
:100FE000822400F582E5833480F583C322900000DB
:100FF000D322C2B6900000D3020FFDC2B6120FB8C2
:10100000E433C0E07537007403125608E51E12562B
:1010100008E51F1256087453125608D0E0125608FD
:1010200074001256087400125608E583125608E53B
:1010300082125608E53712560874FF125608309986
:10104000FD12965922C2B6E5356004F4FF8004FF14
:10105000120D947537007403125608E51E125608D7
:10106000E51F1256087456125608EF125608E53757
:1010700012560874FF1256083099FD1296592274C0
:1010800001C0E0788C75F008E4F608D5F0FBD0E0FC
:10109000D322120FB840E860E878908683088682F1
:1010A0001210A5C322C082C083E58275F008A4F5A2
:1010B00082E5F0C58375F008A42583F583E5F03457
:1010C00004F55EE5822400F582E5833400F5835063
:1010D00002055E7408F9748CF8855E2F858330856F
:1010E0008231120539D083D08222120FB87F085086
:1010F00005120D947F00788E865208865308865418
:10110000088655C2B67537007403125608E51E12DC
:101110005608E51F1256087454125608E535125643
:1011200008EF125608E535603CE5556553F5F0E5E6
:1011300054655245F0600B8555828554831210A585
:101140008003121081855582855483A3120DB285C8
:101150008255858354788C75F008E612560808D5B8
:10116000F0F8D535C4E53712560874FF125608302A
:1011700099FD129659C322E5357007C2AF120FB818
:101180005005E535F4800C7890A65408A655120F4A
:1011900068E535D2AFC0E0C2B675370074031256A9
:1011A00008E51E125608E51F125608745512560817
:1011B000D0E0125608E53712560874FF1256083070
:1011C00099FD129659D322C2B67537007403125690
:1011D00008E51E125608E51F1256087458125608E4
:1011E000758200E53524CFF5837F107410F9748C77
:1011F000F8752F00858330858231120539788C7E11
:1012000010E612560808A3DEF8DFE0E537125608AC
:1012100074FF1256083099FD129659D3221278960F
:101220007892E630E402240A540FC4F97891E6C4B7
:10123000540375F00AA4F5F0E6540F25F0C31349E2
:10124000788DF67891E692E754C0F9788FE6C45429
:101250000775F00AA4F5F0E6540F25F049F97890E7
:10126000E6C4540375F00AA4F5F0E6540F25F0F532
:10127000F0788EE654702345F0788FF6788EE9F694
:1012800022E4305D0978BDE2600378BEF2221212DA
:10129000B6E450F978BDE260F478BFF2221212B6DB
:1012A00050EB78BFE2C36005D2597401F2D32278C3
:1012B000C0E278BFF22220380A30370778C0E260F7
:1012C00002D322C322A206B392A5A207B392A7A279
:1012D00008B392A6AC803039068C804380EF22752B
:1012E000801F00000000E58075807F540FB40F035D
:1012F000021323E5807580BF30E03130E13D30E2FC
:101300004930E355E5807580DF30E02530E131304C
:10131000E23D30E313E58030E01C30E12830E23478
:1013200030E33B74FF02136BE402136B740102138E
:101330006B740202136B740302136B740402136B5D
:10134000740502136B740602136B740702136B743B
:101350000802136B740902136B740A02136B740B8B
:1013600002136BF53C753D010212D9B53CF5D53D34
:10137000F7B4FF030212D9F53ED2390212D9C29056
:10138000C2AFA284D284C0D0C284D290C290A295AF
:10139000B39203D290C290A295B39204D290C2901D
:1013A000A295B39205D290C290A295B3D290C2906A
:1013B000A295B3D0D09284D2AFD290223039FD1210
:1013C000700C75F00612011D12701375F0141201E5
:1013D0001DE53EC23922C0E0E56E5420600AD0E02F
:1013E0006003B4090874FF22D0E0D25122B4010591
:1013F00074BCD25022B4020574BDD25022B403058D
:1014000074BED25022B4040574BFD25022B4050574
:1014100074BCD25122B4060574BDD25122B4070562
:1014200074BED25122B4080474BFD25122788C7990
:1014300010E6B5F0070805F0D9F7E422740122C0E0
:10144000E0788C7910F60805E0D9FA7410F9748CFC
:10145000F8752F037530FA7531001204C67410F94F
:10146000748CF8752F037530FB7531001204C67447
:1014700010F9748CF8752F037530FA753100120568
:1014800039D0F0C0F012142D701E7410F9748CF85D
:10149000752F037530FB753100120539D0F0C0F09F
:1014A00012142D7003D0F022D0F022E51DC0E012FE
:1014B000143FD0F07006E5F0F412143F22788B74DC
:1014C000FFF21218E4C2121209346001221206B7A8
:1014D0007401F9748BF8752F01753000753110C0E7
:1014E000F01204F7D0F07401F974B2F8752F017599
:1014F0003000753111C0F01204F7D0F07401F974A6
:10150000B3F8752F01753000753113C0F01204F770
:10151000D0F07402F9749AF8752F017530007531A6
:1015200070C0F01204F7D0F07416F974C2F8752F79
:1015300001753000753140C0F01204F7D0F078C268
:101540009000D875F016E2F008A3D5F0F97416F9FA
:1015500074C2F8752F01753000753120C0F0120487
:10156000F7D0F07408F97400F8752F017530047520
:101570003100C0F01204F7D0F0780090020375F04B
:1015800008E2F008A3D5F0F9900208E0B4FF14A334
:10159000E0B4FF0FA3E0B4FF0A9002087483F0A345
:1015A000F0A3F0D212E42212160812167D22788CD3
:1015B00076457401F9748CF8752F0275308E75318B
:1015C000001204C6788C76457401F9748CF8752F76
:1015D0000275308E7531081204C622788C76AC7490
:1015E00001F9748CF8752F0275308E753100120474
:1015F000C6788C76AC7401F9748CF8752F0275304E
:101600008E7531081204C622788C76FF08E4A23861
:1016100092E0A23792E1F67402F9748CF8752F0209
:1016200075308E7531001204C622D262D238D2379C
:10163000C2637402F9748CF8752F0275308E75319F
:1016400000120539788CB6AC028009B64518E56FF2
:101650005401601208E6A2E09238B39263A2E192CC
:1016600037757A1FC262788C76FF7401F9748CF832
:10167000752F0275308E7531001204C622788C7673
:10168000FF08E4A24F92E0A24E92E1A21592E2A2DC
:101690000792E3A20892E4F608A64908A64A087948
:1016A0007EE7F608A67508A67408E4A26792E0A291
:1016B0006892E1A26592E2A26692E3F608740012D3
:1016C0007EB2E492E0C0E07401127EB2D0E092E11A
:1016D000C0E07402127EB2D0E092E2C0E074031265
:1016E0007EB2D0E092E3C0E07404127EB2D0E09209
:1016F000E4F608A64F08797DE7F674FF08A66808A7
:10170000A66908F608F608E4A22292E0A22392E174
:10171000A22492E2A22092E4A21F92E5A21492E6F1
:10172000F67410F9748CF8752F0275308E753108C7
:101730001204C6223012487883E6604354016005E3
:10174000D262120A57D21E7883E654026003126EE8
:10175000837883E654046003126DD77883E65408D7
:101760006003127E527883E6541060031267E878B3
:1017700083E654206003126D86C21E7883760022B1
:101780007410F9748CF8752F0275308E753108124B
:101790000539D21E788C7F00B6AC107F01800F789F
:1017A0008376FE1217347F020218CDB645F1EF7032
:1017B00011E56F5404700BEFC0E0126DD7D0E0FF5D
:1017C000802F788DE6A2E0924FA2E1924EA2E392A2
:1017D00007D26AA2E49208754900754A00304E0BA0
:1017E000A2E29215788E864908864A7890E6797E3C
:1017F000F7EF7011E56F5402700BEFC0E0126E83CB
:10180000D0E0FF80197891867508867408E6A2E01A
:101810009267A2E19268A2E29265A2E39266EF70FB
:1018200006E56F5408603A7894E6A2E0C0E07400E0
:10183000127E67D0E0A2E1C0E07401127E67D0E0C2
:10184000A2E2C0E07402127E67D0E0A2E3C0E074BE
:1018500003127E67D0E0A2E4C0E07404127E67D079
:10186000E0EF7013E56F5420700DD21EEFC0E01250
:101870006D86D0E0FF80097895864F08E6797DF780
:101880007897866878988669EF700FE56F541070C6
:1018900009EFC0E01267E8D0E0FFD228EF602EC267
:1018A000287897E67898E67899E6789AE6789BE63D
:1018B000A2E09222A2E19223A2E29224A2E4922048
:1018C000A2E5921FA2E6921412856B9216788C768E
:1018D000FF7401F9748CF8752F0275308E7531081C
:1018E0001204C62278C275F016E4F208D5F0FB7433
:1018F000FF78CAF278CBF2227403F97495F8752F49
:101900000075308C7531E5C0F01204F7D0F0789591
:10191000E224FD920EE224E2920F7401F97494F82D
:10192000752F0075308C7531E2C0F01204F7D0F0DD
:10193000227403F97495F8752F0075308C7531E5B4
:101940001204957401F97494F8752F0075308C7534
:1019500031E212049522798C770309774D097703D8
:101960000977040977060977027406F9748CF8750B
:101970002F0075308D7531201204C67406F9748CF1
:10198000F8752F0275308D7531201204C62274044B
:10199000F9748CF8752F0075308D7531201205396A
:1019A000798EE7640322E4A22592E0A22692E1A2C6
:1019B0002792E2798CF77401F9748CF8752F007511
:1019C000308C7531E81204C6227401F9748CF875F4
:1019D0002F0075308C7531E8120539798CE7A2E05B
:1019E0009225A2E19226A2E2922722798CE4A229F2
:1019F00092E1A22A92E2A21C92E392E492E5A22C46
:101A000092E692E7F709E4A22B92E0A22D92E1A2DE
:101A10002E92E6A22F92E7F709E4A23092E0A232DA
:101A200092E2A23392E3A23492E4A23592E5A23686
:101A300092E7F709E56AF77404F9748CF8752F00DA
:101A400075308C7531EC1204C6798CE56BF4F709AE
:101A5000E56CF4F709E56DF4F77403F9748CF87527
:101A60002F0075308C7531E91204C6798CE56EF45F
:101A7000F709E56FF4F709E570F4F77403F9748C6E
:101A8000F8752F0075308D7531041204C622740468
:101A9000F9748CF8752F0075308C7531EC1205399E
:101AA000798CE7A2E19229A2E2922AA2E3921CA2F7
:101AB000E6922CA2E709E7A2E0922BA2E1922DA2E6
:101AC000E6922EA2E7922F09E7A2E09230A2E292DC
:101AD00032A2E39233A2E49234A2E59235A2E6A2C6
:101AE000E7923609E7F56A7403F9748CF8752F00EC
:101AF00075308C7531E9120539798CE7F4F56B098D
:101B0000E7F4F56C09E7F4F56D7403F9748CF87576
:101B10002F0075308D753104120539798CE7F4F595
:101B20006E09E7F4F56F09E7F4F57022798CF77424
:101B300001F9748CF8752F0075308C7531E412043E
:101B4000C6227401F9748CF8752F0075308C7531CC
:101B5000E4120539798CE7227881E270067882F206
:101B600008F22275F00030340475F03CA4AAF07538
:101B7000F008A4FBACF0EA75F008A42CFAC3E49BCF
:101B8000FBE49A7882F2EB08F2227401F9748CF883
:101B9000752F0075308C7531F01204957401F9744D
:101BA0008DF8752F0075308C7531F4120495740121
:101BB000F9748EF8752F0075308C7531F612049516
:101BC0007401F9748FF8752F0075308C7531F2122D
:101BD0000495227401F9748CF8752F0075308C759A
:101BE00031F0C0F01204F7D0F07401F9748DF8757B
:101BF0002F0075308C7531F4C0F01204F7D0F074FA
:101C000001F9748EF8752F0075308C7531F6C0F0BF
:101C10001204F7D0F07401F9748FF8752F00753045
:101C20008C7531F2C0F01204F7D0F0227401F9740F
:101C300038F8752F0075308C7531F91204C67401AF
:101C4000F97439F8752F0075308C7531F81204C6A7
:101C50007401F9743AF8752F0075308C7531FA12E9
:101C600004C6227401F97438F8752F0075308C752C
:101C700031F91205397401F97439F8752F0075308E
:101C80008C7531F81205397401F9743AF8752F0022
:101C900075308C7531FA120539227402F9741EF808
:101CA000752F0075308C7531E01204C6227402F96C
:101CB000741EF8752F0075308C7531E012053922CD
:101CC000E56D5402600375641878A57990E5647534
:101CD000F00484FAC0F080021819E7F5F066540F9A
:101CE0007036DA0CD0E0602EFA18E7C4F5F08016F2
:101CF00018E7C4F5F066540F701EDADCD0E0601609
:101D0000FA1819E7F5F0E4D333DAFCFAE65AC5F02D
:101D10005AC395F0700EE422D0E0E6540FC5F0549B
:101D20000FC395F09211740122789179947A03E6A9
:101D3000C4540FF709E6540FF70908DAF2799478DA
:101D4000A87A06E6540FF6E76670080908DAF4E4A4
:101D5000C23B22799978AD7A06C3E7961918DAFA68
:101D60009211799978AD7A06E7540FB40F08E654CA
:101D70000FB40F108008E6540FB40F0B800618192B
:101D8000DAE680CB740122C3E796B409028012140C
:101D9000600FC3E7F5F0E695F0B409028003147014
:101DA000E3E9B49404E4D23B221918E766540F60C7
:101DB000F080D1121D29701F303B1C202B1AC2AF9E
:101DC00075185085831985821A12972375710074CE
:101DD00005127E69D23AE42204227408F9748CF860
:101DE000752F0075308C7531C0120539121CC02258
:101DF0007408F9748CF8752F0075308C7531C01229
:101E00000539121DB322E58275F008A42420F5825D
:101E1000500205F0A8F0E58375F008A4282400F529
:101E20008322C082C083121E067408F9748CF87570
:101E30002F00858330858231120539D083D082020C
:101E40004FB6751B20751C009000007405F9748C4A
:101E5000F8752F00851C30851B31120539121CC006
:101E60006018E51B2408F51B5002051CA3E583B48C
:101E700003D9E582B4E8D4740122121E22E4229030
:101E80000000121E22121CC022751B00751C00755A
:101E90005C9F755B0F80153012E5E570540270A2EF
:101EA000751B00751C00755C9F755B0FE55C251B41
:101EB000C2E0F582E55B351CF583C082C083E58214
:101EC0002400F582E5833425F5837402F9748CF8D7
:101ED000752F01858330858231120539788C868390
:101EE000088682121E22121CC07005D0F0D0F0228B
:101EF000D083D082C3E58313F583E58213F5822076
:101F00001114E58245836022E58224FFF55CE583B8
:101F100034FFF55B8007A385821B85831CC3E55CCA
:101F2000951BE55B951C4002808274012230123AB9
:101F30007410F9748CF8752F0175300075316012CA
:101F40000539789C798C75F00AE7B4FF02801BB4E0
:101F50003C130809D5F0F2900FE878D0E27887F2C8
:101F60007886F2E42266540F60E8740122751B251E
:101F7000751C009000007403F97491F8752F0085AA
:101F80001C30851B31120539121DB36018E51B2466
:101F900008F51B5002051CA3E583B403D9E582B400
:101FA000E8D4740122121E22E422900000121E22A4
:101FB000121DB322751B00751C00755C9F755B0FAD
:101FC000802078A8E6540FB40F030220603012DAA4
:101FD000E57054027097751B00751C00755C9F7549
:101FE0005B0FE55C251BC2E0F582E55B351CF583E4
:101FF000C082C083E5822400F582E5833445F58301
:102000007402F9748CF8752F018583308582311242
:102010000539788C8683088682121E22121DB370C1
:1020200005D0F0D0F022D083D082C3E58313F583AE
:10203000E58213F582201114E58245836022E58252
:1020400024FFF55CE58334FFF55B8007A385821BE5
:1020500085831CC3E55C951BE55B951C4002808273
:1020600074012230410DE536B44308E53424FE50B6
:102070000280F0789C7A0579B0E6540FC4F5F00838
:10208000E6540F45F0F70809DAEF22120093129791
:102090000D75F00F129625D5F0FA30A0EE22D21D64
:1020A000D2A3C248C2A2D24BD2A1C24AD2A4C24930
:1020B00012208B12970D12703C40F81266211224E8
:1020C0002E1264C4127819120D941206F9C2A3C21A
:1020D00048C2A2C24BC2A1C24AD2A4C2490274677A
:1020E000D2A3C248C2A2D24BD2A1C24AD2A4C249F0
:1020F000754E001233E11233F712703C5002809E8D
:10210000D21D12208BD21D12797F12651E400C1237
:10211000234D1264C4120D941206F9027467C2A30F
:10212000C248C2A2C24BC2A1C24A1270131222DC20
:102130004050C01D1208D0D0F07047E51D95F078D2
:10214000B6F212222D12198E601AD21D90000012C2
:102150001E2212234D1264C4120D941206F9129716
:102160000D12222D1214BD12256F401FE56D54086B
:10217000700F1277EA500712797F1221EC22127940
:102180005E2212256F789DE24402F212797FD2A37B
:10219000C248D2A2C24BC2A1C24AD2A4C249C21DE5
:1021A0007548FA12421675F064129625D5F0FA12A7
:1021B000421675F064129625D5F0FA12700C124290
:1021C0001675F064129625D5F0FA12421675F06471
:1021D000129625D5F0FA12701312703C50030220AB
:1021E0009E12749E50A80220E0020000D2A0129617
:1021F0004130A0F5D2A3C248D2A2C24BC2A1C24A6A
:10220000D2A4C249C21D7548FA75F014129625D59C
:10221000F0FA12700C75F014129625D5F0FA1270BF
:1022200013126C061242161277EA40C0221219C924
:10223000121A8E121B42A2E49265A2E59266A2E6F1
:102240009267A2E792687401F97481F8752F00759E
:10225000308C7531FCC0F01204F7D0F07401F974C1
:1022600084F8752F0075308D753100C0F01204F7B9
:10227000D0F0121BD3121C637401F974BCF8752FD3
:1022800001753000753173C0F01204F7D0F078BCDE
:10229000E2B4FF02E4F27401F974BDF8752F017520
:1022A0003000753174C0F01204F7D0F078BDE2B49C
:1022B000FF02E4F27401F974C0F8752F0175300063
:1022C000753175C0F01204F7D0F078C0E2B4FF02A7
:1022D000E4F2121CAD1218F8121B58227410F97493
:1022E0008CF8752F0075308C7531E0120539788CBB
:1022F000E6B430004053B43A00504E08E6B4300023
:102300004047B43A0050427A10788CB6FF3D08DA64
:10231000FA7410F9748CF8752F0075308C7531F0E3
:102320001205397A10788CB6FF2108DAFA7410F9A0
:10233000748CF8752F0075308D7531001205397A5F
:1023400010788CB6FF0508DAFAD322C322D21DC258
:10235000A3C248C2A2C24BC2A1C24AD2A4C249C0AF
:102360001EC01F788C9000007A08E6F008A3DAFA05
:1023700012242E127819788C9000007A08E0F60862
:10238000A3DAFA7408F9748CF8752F0075300075AB
:1023900031201204C67408F9748CF8752F0075305A
:1023A0008C7531C01204C6D01FD01E121C9A227523
:1023B0001E30751F3012252ED225C226C227C229F3
:1023C000C22AC21CC22CC22BD22DC22EC22FC23096
:1023D000C232C233C234C235C236756A00756B0070
:1023E000756C00756D08756E00756F00757000C2B4
:1023F00065C266C267C26878817404F27884740921
:10240000F2788C7401F2788D7402F2788E7404F292
:10241000788F7404F2753863753907753A00740162
:102420007894F27895F2E408F208F2C212221209C6
:10243000751223AF121C9A1219A61219EBC2E0A250
:102440006592E4A26692E5A26792E6A26892E7121C
:102450001B2C7401F97481F8752F0075308C75315F
:10246000FC1204957401F97484F8752F0075308D91
:10247000753100120495121B8A121C2C121931128C
:1024800019561267E822E5822420F582E583347D1F
:10249000F5837401F97488F8752F0085833085827F
:1024A00031C0F01204F7D0F07888E222C0E0E58273
:1024B0002420F582E583347DF583D0E07888F274BA
:1024C00001F97488F8752F008583308582311204F4
:1024D00095227401F97498F8752F017530007531E3
:1024E000721205397898E6B4FF02740522746E8082
:1024F0000712250E501774FF789CF27401F9749C32
:10250000F8752F0275308E753138120495227401DA
:10251000F9749CF8752F0275308E753138C0F01241
:1025200004F7D0F0789CE2B46E02D322C322C082BA
:10253000C083909BBBE493B430004026B43A005073
:1025400021F5F0A3E493B430004017B43A005012E0
:1025500085F01EF51F90009DE04401F0D083D082ED
:10256000D32290009DE054FEF0D083D082C322128B
:1025700079DE400E788CE6B51E1308E6B51F0E1204
:102580007A0212252E789DE254F7F2C322788C86C7
:102590001E08861F789DE24408F2127A0212252E48
:1025A000D3222643266F26B5261726172617261769
:1025B00026DE26E926F426FF270A2745273F277C23
:1025C0002794279F27F32854287228A228C928E493
:1025D00028FF29082923293E29472962297D2986A0
:1025E00029A12C142C4A78B9E224DE402A122B4B64
:1025F000401378B9E225E0049025A293C0E0E225DB
:10260000E093C0E022022C0778B9E2122C04122CCD
:10261000061200D6024D24740A022C07D2A1C24A27
:10262000C2A4D249122C051200E3122FF720430254
:10263000D322E53BB402F978A8E624F640F208E696
:1026400024F622C01EC01F12252ED01FD01E401AF5
:1026500012261C401578A8E62430F51E08E6243022
:10266000F51F121C9A1264C4809E7420022C07125B
:102670002AE4403C12789678A8E6C40846F5F0C0F3
:10268000F078ACE675F00AA408267893F6540303B4
:1026900003D0F045F07891F678AAE6C40846F5F044
:1026A00078AEE6C42345F07892F612783202260816
:1026B000741E022C07122A95401F12789678A8E6FD
:1026C000C408467890F678AAE6C40846788FF6E4FF
:1026D000788EF6127832022608741F022C07122B0D
:1026E000E5741B1283DA022608122BE5741B128391
:1026F000FB022608122BE5741B12843D02260812E9
:102700002BE5741B12841C022608122BE51254DDE3
:10271000C238757A1FD263787FE2F58308E2F582CA
:10272000C2AF75186085831985821A129723121219
:10273000AF1255A37573030226087416022C0720E6
:1027400038C802274512855040F012856240EBC21E
:1027500063122BE5120C7AD238757A1F787FE2F576
:102760008308E2F582C2AF75187085831985821AD5
:10277000129723125594757303022608122BE51243
:1027800015A71215AE75F0C8129625D5F0FA126D80
:102790002F027467122BE5741B1284D5022608E5FC
:1027A000796003B4020F122C05C079122A5BD0792C
:1027B000403C78BAF278BAE2F54F7899F2122BE5FC
:1027C000C2AF751830854F1A751903E579600C781A
:1027D000BBE2F519B40504C250C251431900129767
:1027E00023E57960061200D6024D24022608741AE9
:1027F000022C07E5796003B4020F122C05C0791290
:102800002A5BD07940E878BAF278BAE2F54F122B19
:10281000E5C2AF751830854F1A751903E57960095F
:1028200078BBE2F519C250C251431908129723121E
:102830006C06126C40124E29D2A2C24BC2A1D24ADF
:102840001200E3122FF7741820420620430330448D
:102850009F02463C1212816044122BE5741B543FC8
:102860004480C2AF7518C0751909F51A1297230272
:102870002608305D14122C05122A5B40076023786D
:10288000BEF280D5741C022C071212B6500F122C07
:1028900005122A5B40EE602A78BFF280BC741D02EC
:1028A0002C07305D1DE478BEF2122BE5741B543FFB
:1028B0004440C2AF7518C0751909F51A1297230262
:1028C000260812129D50D680E07400127E69741B97
:1028D000543F4400C2AF7518C075190AF51A129713
:1028E000230226087400127E95741B543F4480C254
:1028F000AF7518C075190AF51A12972302260874C5
:1029000000127EB240DE80C17402127E69741B54D4
:102910003F4400C2AF7518C075190CF51A12972301
:102920000226087402127E95741B543F4440C2AFC5
:102930007518C075190CF51A12972302260874022F
:10294000127EB240DE80C17403127E69741B543F54
:102950004480C2AF7518C075190CF51A129723027E
:1029600026087403127E95741B543F44C0C2AF7591
:1029700018C075190CF51A12972302260874031251
:102980007EB240DE80C17404127E69741B543F44E1
:1029900040C2AF7518C075190BF51A12972302269D
:1029A000081296F3741B543F4480C2AF7518C0756B
:1029B000190BF51A129723022608C2A1D24AC2A403
:1029C000D249124E291200E3122FF7204409204267
:1029D0001F2043510229EE787FE2F58308E2F58259
:1029E000120101301206124FB620E202C322D32296
:1029F000121E9770F912557EB4020280F1B4031AC8
:102A0000C082C0831200E3122E04D083D0823043F0
:102A1000DDE53B60D9121DB370D4787FE583F20801
:102A2000E582F280BB121FC270C412557EB401024F
:102A300080BCB40324C082C0831200E3122FF7D0FD
:102A400083D0823042A8C082C08312010112206369
:102A5000D083D082121CC0709580BFD2A1C24AC25E
:102A6000A4D2491200E3122FF7204302D322E53B00
:102A700060FA24FC40F6A93B78A87A00B60A005018
:102A8000EBEA75F00AA42640E3C5F070DFAAF0086F
:102A9000D9EAEAC322D2A1C24AC2A4D249122C0561
:102AA0001200E3122FF7204302D322E53BB404F9CE
:102AB000F5F078A8E624F640F008D5F0F778A8E617
:102AC00075F00AA4082624E8402E78AAE675F00AD4
:102AD000A4082624C4402122E0E2E0E1E0E1E0E0B5
:102AE000E1E0E1E0D2A1C24AC2A4D249122C05120F
:102AF00000E3122FF7204302D322E53BB407F9F598
:102B0000F078A8E624F640F008D5F0F778AAE67544
:102B1000F00AA4082660E1C0E024F3D0E040D99098
:102B20002AD793F978A8E675F00AA4082660C9C0E8
:102B3000E029D0E040C278ACE675F00AA40826246B
:102B40009C40B578AEE624F940AE2230127D787F05
:102B5000740FF20874E9F2E579707C78B9E2240028
:102B6000F5827583027401F9748CF8752F018583E1
:102B700030858231120539788CE61201595062781D
:102B8000B9E22400F5827583037401F9748CF87539
:102B90002F01858330858231120539788CE6120148
:102BA000A9503678B9E22400F5827583017401F9E1
:102BB000748CF8752F018583308582311205397840
:102BC0008CE620500C20E01530E10C1229BA740D6F
:102BD0002220E20920E3F4C322740E8006740C80E4
:102BE00002740BD322E579701A1233F8787FE2F57C
:102BF0008308E2F582C2AF7518E085831985821AD1
:102C000012972322222222C0E0126E65D0E0120029
:102C1000AA024D24D2A1C24AC2A4D249122C051242
:102C200000E3122FF730431EE53BB4011978A8E604
:102C300054FC7012E60303441CC0E0122BE5D0E004
:102C40001293D1022608742280BDD2A1C24AC2A426
:102C5000D249122C051200E3122FF730431EE53B38
:102C6000B4011978A8E654FC7012E60303441CC0B2
:102C7000E0122BE5D0E01293E70226087422808749
:102C8000304C19C24C306E1D128550500AC2A3D26E
:102C900048C2A4D249800E126E77800975F00C20CC
:102CA000B305D5F0FAD322C322201D31E8C0E0E9F4
:102CB000C0E0EAC0E0200E26122C805017122F9799
:102CC000754E007895E2600C75F003129625D5F0EC
:102CD000FA12324AD0E0FAD0E0F9D0E0F822200F20
:102CE000133056F0C082C083122D0B127AD6D083D7
:102CF000D08280E03056DDC082C083E5637003126D
:102D00002DB7127C47D083D08280C9D250C251786F
:102D100095E2B40F0B127C065003022DAF022D4931
:102D2000B41010127C065003022DAF125133D2435F
:102D3000022DB6B4110B127C064074125044022DC1
:102D40006CB4030D127C0640661251BED243022DB4
:102D5000B6B4040D127C0640561250DCD242022D4D
:102D6000B6B40518127C0640461250684041787F80
:102D7000E583F208E582F2D244022DB6B4120512C0
:102D80007C128099B41305127C12809FB41705122F
:102D90007C1280A7B41405127C1280ADB415051204
:102DA0007C1280B5B41605127C1280BD022DAFC214
:102DB00050C251127AD622D250C2517895E275F0A3
:102DC0000384E5F0B400091253C24033D243802F8C
:102DD000B4011CE2B42203206C091253F34020D248
:102DE00042801C127CA44017753B06D2438010120F
:102DF00053F6400B787FE583F208E582F2D2442255
:102E0000D2458005C245122E76757900D24C7548A0
:102E1000FA7440301D02740CF546C243C239E546CF
:102E2000603F122CA920433975F003129625D5F086
:102E3000FA120273201D04E579701A3039E0D2517C
:102E400020451E7546601213BCB40B0D75F00812B8
:102E50009625D5F0FAD2438008122E697548FA807B
:102E6000BDC242D2AF7548FA22533B07F8E53B2476
:102E7000A8C8F6053B2278A875F00874FFF608D5B7
:102E8000F0FB753B002230011BC082C08390028B97
:102E900075F00A74FFF0A3D5F0FB9002977404F06C
:102EA000D083D08222200102E4227A00C082C08333
:102EB00090028B789C75F00A7B00E670010BE0664F
:102EC0006004E6F07A0108A3D5F0EFD083D082BB8E
:102ED00007005002E422C082C0839002977403BAB4
:102EE0000003E015E0F0D083D08222D297122EF5B5
:102EF000C297122EF522C297C2B5122EF5D29712A2
:102F00002EF5D2B5122EF5C297122EF575F00833B4
:102F100092B5122EEBD5F0F722D2B775F008D29702
:102F2000122EF5A2B7C297122EF533D5F0F022C2B9
:102F300097C2B5122EF5D297122EF5D2B5122EF5F4
:102F4000C297122EF5D2B5122EEB122EEB122EEBEB
:102F500022D297D2B77473122EF6744B122EF674D7
:102F600050122EF61296717408122EF6122F192393
:102F7000243F3019022420543F4480122EF6746BF3
:102F8000122EF61296417468122EF6129671746023
:102F9000122EF6122F2F22C2ABC28ED2AFD297D2F0
:102FA000B722C2ABC28ED2AF7455122EF6D297D2D0
:102FB000B722C2AFC28E53890F438910758BD67565
:102FC0008DFBC28FD28ED2AFC23FD2BBD2AB303FCD
:102FD000FD22C0D0A2B7923ED23FD0D0C2ABC28EAB
:102FE000C28F758BEB758DFDD28EC2AF32D245800C
:102FF00008C24574108009C2457440301D0274082F
:10300000F546D24C757900D2217548FA122E76C257
:1030100043C242C239C244122E86C24612027320F3
:103020001D07E5796003023099B20C300C1DB20D1A
:10303000300D18122F97B219D221201D0E122CA973
:10304000204358204255204452D221303960789490
:10305000E27004C2398057754660122F97D2213032
:103060004504D25180351213BC1213D6B4FF02802E
:103070003DB4BC0A123714E5796020023099B4BD22
:103080000280F1B4BE0280ECB4BF0280E7B40B153D
:1030900075F008129625D5F0FAD243757103122FF8
:1030A000977548FA22122E697548FA757103E5463C
:1030B00060EC30210FC2217894E27005122FA280BB
:1030C00003122F51C28EC2ABD2AF20B7063046FAE0
:1030D00002301A12027330B7063046FA02301A79FB
:1030E00008122FB2303EDD208FDA20B7FAD9F278FD
:1030F0009C790B7B007A057C00C23D122FB2208F99
:10310000C320B705203E0580F5203EF2A23E5002C6
:10311000B23DEC33FCDAE4D91A20E0A803540F6B7B
:10312000600280A0122EA5709BD242756428D251F5
:1031300002309B303D0720E0028089808703540FD6
:10314000F6086BFB80AFB40207204307C242C244BB
:103150000231D4C082C08390EA60E53B606324FB07
:10316000405F78A8E6540F758300F582D53B028056
:103170005075F00AA4F58275830008E6540F258285
:10318000F582D53B02803AE58275F00AA4F5828586
:10319000F08308E62582F58250020583D53B028044
:1031A00020E58275F00AA4F582C0F0E58375F00A87
:1031B000A4D0F025F0F58308E62582F582500205BB
:1031C00083787FE583F208E582F2C243C242D244AB
:1031D000D083D08222C0F075F0FAD5F0FD75F0648E
:1031E000D5F0FDD0F0221231D51231D51231D512E1
:1031F00031D51231D51231D522D2B4C29475F00531
:1032000012964120B30612964130B303D5F0F11265
:10321000964122C0F075F008A2E7B39294C2B412AE
:1032200031D5C294D2B41231D5C0E0E430B3010438
:103230000030B301040030B30104D36003D5E001D2
:10324000C3D0E033D5F0D1D0F022D2B4C294D2B3FF
:103250001231D5C2B41231E6D2B41231E6201D03C8
:1032600030512378847601087480F608A2A3B392C3
:10327000E4F6749008F608F608F608F60232DB78F1
:1032800084760502328A7884760308768008748012
:1032900030480C304909207408D274D24C800FC2D7
:1032A00074A24892E5A2A3304901C3B392E4A24BB1
:1032B00092E1201D04A21592E0F6087480201D12F0
:1032C00020510FE54E54074480A24A92E5A2A1B3D3
:1032D00092E4F6087480F608F608F675F00778842C
:1032E0007E007F00E62EFEE6123213F62FFF08D591
:1032F000F0F2EED333123213F8EFD33368707278F2
:1033000084B6FF6D0557E55724FE50167557022009
:103310001F10D21FC2AF7518C0751900751A03129D
:103320009723201D087895E260033051030233DDB6
:10333000788AE620E37120E26120E1547885E6B6E0
:10334000002D08B6421508E6A250C0D0D250123760
:1033500014D0D0306F0292500233DDB6551108B64A
:10336000000D08797FE6F30809E6F3D244D25080D5
:103370006CE5576019D55716301F13C21FC2AF75C1
:1033800018C0751900751A04129723757203804DC1
:10339000D2507885863ED23980437885863B08D2E4
:1033A0004379A87A04800B7885D242756428799C89
:1033B0007A05D25075F00FE6C4540FF755F0F5F0CA
:1033C00009E6540FF755F0F5F00908DAEAE5F0B42C
:1033D0000F051977EEC2427895E21231461231F9A3
:1033E000227895E2601024FD400C75F003129625BA
:1033F000D5F0FA12324A2222C0E030500EC2AF7528
:1034000018B0751900751A00129723D0E0D26F22F8
:10341000D2B4C294D2B31231D5C2B41231E6D2B40E
:103420001231E67884E567540FC44407F608E56670
:1034300023A2E392E5A2E292E3542AD2E6D2E7F68F
:1034400008E566A2E392E1A2E492E3542AD2E6D22E
:10345000E7F608E566A2E692E1A2E792E3540AD213
:10346000E6D2E7F674C008F608F608F675F00778B5
:10347000847E007F00E62EFEE6123213F62FFF0850
:10348000D5F0F2EED333123213F8EFD33368700B6A
:103490007884B6FF061231F9C380041231F9D322C1
:1034A0001234A950031234A922127AF9E4C0E0754B
:1034B0006708789EE2F566123410740040051235F4
:1034C000DC800A1236044005D0E004C0E0756709CC
:1034D000789FE2F566123410740140051235DC80E5
:1034E0000A1236044005D0E004C0E075670A78A0EF
:1034F000E2F566123410740640051235DC800A12BB
:1035000036044005D0E004C0E075670B78A1E2F511
:1035100066123410740740051235DC800A12360436
:103520004005D0E004C0E012746CD0E0C36001D369
:103530002222E56A542060F97567047566FF12342B
:103540001074025004123604221235DC7887795741
:10355000E6F30809E6F3087959E6F30809E6F37893
:1035600085E6A2E092E25414F5F008E623A2E59283
:10357000E0540345F0F5F0785BE265F0C0E0E5F07B
:10358000F2D0E030E221C0E0C0F0E5F075F0493063
:10359000E20375F04AC2AF7518C075190085F01ABC
:1035A000129723D0F0D0E0540370030235DBE5F02E
:1035B0005403B4030575F0488013B4020575F04751
:1035C000800BB4000575F04B800375F04CC2AF75ED
:1035D00018C075190085F01A12972322F5F0245DA2
:1035E000F8E2B40205227402F22250FA7402F2E503
:1035F000F02432F5F0C2AF7518C075190085F01AC5
:1036000012972322F5F0245DF8E2C3601D14F2D373
:103610007018E5F0243CF5F0C2AF7518C0751900BC
:1036200085F01A129723757203D322D2B4C294D2B2
:10363000B31231D5C2B41231E6D2B41231E6788475
:10364000E567540FC44403F6087680087480A248E6
:1036500092E5A2A3B392E4A24B92E1A21592E0F606
:10366000087480A24A92E5A2A1B392E4F60874809D
:10367000F608F608F675F00778847E007F00E62EDF
:10368000FEE6123213F62FFF08D5F0F2EED3331216
:103690003213F8EFD3336870717884B6FF6C788A90
:1036A000E620E33020E22020E1607885E6B6005A8B
:1036B00008B6551108B6005208797FE6F30809E606
:1036C000F3D244804A80437885863B08D24379A868
:1036D0007A04800B7885D242756428799C7A0575C6
:1036E000F00FE6C4540FF755F0F5F009E6540FF764
:1036F00055F0F5F00908DAEAE5F0B40F051977EEB0
:10370000C2427898E212314680051231F9D3221272
:1037100031F9C322C26FB4FF157562051233F8C2C6
:10372000AF7518C0751900751A0712972322B4BC1B
:1037300003023747B4BD03023779B4BE030237AB87
:10374000B4BF030237DD222050147408F9748CF8DA
:10375000752F01753000753180120539801274089B
:10376000F9748CF8752F01753000753188120539A0
:1037700074117894F612380F222050147408F974DA
:103780008CF8752F01753000753190120539801253
:103790007408F9748CF8752F017530007531981222
:1037A000053974127894F612380F222050147408D8
:1037B000F9748CF8752F017530007531A012053938
:1037C00080127408F9748CF8752F0175300075310A
:1037D000A812053974137894F612380F2220501469
:1037E0007408F9748CF8752F017530007531B012BA
:1037F000053980127408F9748CF8752F0175300042
:103800007531B812053974147894F612380F22788D
:103810008DE61201594004741ED322788EE61201FF
:10382000A9400C741FD322126E771200D6C32278DF
:103830008CE660F9788CE6B4FF06756205023B0001
:10384000B402142032031233F87894E6C2141283BF
:1038500054400280D880D0B404147894E62453C233
:10386000AFF51A7519007518C002972380B9B4090D
:103870001BC0E07404127E69D0E01233F8C2AF7549
:1038800018C0751907F51A129723809BB430087574
:10389000F0041270768096B4310875F004127093BB
:1038A000808BB43808788FE6123B458080B43909A4
:1038B000788FE6123B4B02382DB43A251212816004
:1038C0001D1233F8789486F0E5F0543F4480C2AF7F
:1038D0007518C0751909F51A12972302382702388E
:1038E0002DB43B2B305D21E478BEF21233F878948E
:1038F00086F0E5F0543F4440C2AF7518C075190911
:10390000F51A12972302382712129D50D180DCB489
:103910003C0C1233F87894E61284D5023827B43D73
:103920004B1233F820381ED238757A1FC263C2AFEB
:1039300075187075190F751AE91297231255947539
:103940007303023827C238757A1FD263C2AF751865
:103950006075190F751AE91297231212AF1255A349
:103960007573031254DD02382702382DB43E13E577
:103970006A5410600A1233F8E4123B13023827022B
:10398000382DB43F14E56A5410600B1233F874FFFD
:10399000123B1302382702382DB4400C1233F8784A
:1039A00094E61283DA023827B4410C1233F8789483
:1039B000E612843D023827B4420C1233F87894E6BC
:1039C00012841C023827B4430C1233F87894E612A0
:1039D00083FB023827B444117400127E691233F855
:1039E0007894E612968D023827B445117400127E41
:1039F000951233F87894E612969E023827B4460959
:103A00007400127EB240E580CFB447117402127E7A
:103A1000691233F87894E61296AF023827B4481149
:103A20007402127E951233F87894E61296C002382A
:103A300027B449097402127EB240E580CFB44A111E
:103A40007403127E691233F87894E61296D1023824
:103A500027B44B117403127E951233F87894E61252
:103A600096E2023827B44C097403127EB240E58016
:103A7000CFB44D1D1296F31233F87894E6543F44B8
:103A800080C2AFF51A75190B7518C012972302384A
:103A900027B44E0C3038061233F802394502382765
:103AA000B44F092038F71233F8023927B45412748E
:103AB00000C0E01233F8D0E07894461293E7023861
:103AC00027B45504744080E9B45604748080E2B48D
:103AD000570474C080DBB458127400C0E01233F88D
:103AE000D0E07894461293D1023827B45904744038
:103AF00080E9B45A04748080E2B45B0474C080DB53
:103B00001233F8C2AF7518C0751907F51A1297234A
:103B100002382D789EF208F208F208F2C0E0123462
:103B2000A0D0E07010C2AF7518C0751900751A6981
:103B3000129723C322C2AF7518C0751900751A6A8F
:103B4000129723C32275F00402708375F00402708B
:103B50009A700475591E22D21B22C298C299322033
:103B600075F8201DF5309937C29920411875340039
:103B7000802DD2B6D269C241753400D240D0D0D0A7
:103B8000E0D0F080D5C0F0C0E0C0D0E581240B408B
:103B9000E175D010E534123EA0D0D0D0E0D0F020B6
:103BA000980132C2982041FAC0F0C0E0C0D0E5814F
:103BB000240B40BE75D010304005C240753F00E573
:103BC0004324FE4003754302E53F20E72420E61E20
:103BD000E53F540723246EC0E0E4343DC0E0E5999E
:103BE00022053F2542F542D0D0D0E0D0F032024449
:103BF00018543F2323246FC0E0E4343CC0E0E5992F
:103C000022155880DC80DAD558FBB5420ED21A88CE
:103C1000F0126CFEA8F0753F0080CC023D7EB462CD
:103C2000FA80BE80BCB42AF380B7F55824C6E558A4
:103C300040E924F5E55850E3055880A57850F21581
:103C400058809E7851F2155880977852F215588016
:103C5000907853F2155880897854F21558808278FC
:103C600055F21558023BE17856F21558023BE10235
:103C70003DA200023C1E00023C2300023C25000243
:103C80003C2A00023C0100023C0100023C0100020F
:103C90003C0100023C3C00023C4300023C4A000262
:103CA0003C5100023C5800023C5F00023C670002AD
:103CB0003C0700023C0700023C0700023C070002F0
:103CC0003C0700023C0700023C0700023C070002E0
:103CD0003C0700023C0700023C0700023C070002D0
:103CE0003C0700023C0700023C0700023C070002C0
:103CF0003C0700023C0700023C0700023C070002B0
:103D00003C0700023C0700023C0700023C0700029F
:103D10003C0700023C0700023C0700023C0700028F
:103D20003C0700023C0700023C0700023C0700027F
:103D30003C0700023C0700023C0700023C0700026F
:103D40003C0700023C0700023C0700023C0700025F
:103D50003C0700023C0700023C0700023C0700024F
:103D60003C0700023C0700023C0700023DA2800E17
:103D70008039803D804180448047805B8059B40910
:103D800009754200753F00023BE1B421097542000C
:103D9000753F40023BE1B44209754200753F800225
:103DA0003BE1754200753F00023BE7B51ED0023B88
:103DB000E1B51FCA023BE1F540023BE1F541023BA0
:103DC000E1B542BA75432088F0126CFEA8F0123DAE
:103DD000D9753F00023BE780C985403612729FD2F9
:103DE00041E536B44610E5416003023E9612724D3D
:103DF000C24175651122B447041272B522B4500C49
:103E000085413512724DC24175650722B453108544
:103E10004135E541700812724DC24175650222B408
:103E2000540C85413512724DC24175650122B4555D
:103E30000C85413512724DC24175650322B4560C92
:103E400085413512724DC24175650422B4570C8507
:103E5000413512724DC24175650522B4580C854139
:103E60003512724DC24175650622B44E1F8541352B
:103E7000E541B4010912724DC24175650922B402CF
:103E80000912724DC24175650E22E53624BF24E643
:103E9000400485413522C24122C5372537C5372226
:103EA000E53424F0400DE5342324BEC0E0E4343E84
:103EB000C0E022759906C241753400D2B622802F27
:103EC0008034803680388039803E804680488051FA
:103ED000804F804D804B80468050800E023F5B7546
:103EE0003403F599123E99053422E535023F1475E5
:103EF0003700740380ECE51E80E8E51F80E4023F94
:103F0000C1E53775340F80DA129772123B5188354C
:103F100080D0E53580C9E535A23892E080C175349E
:103F200003A8350535E676FF80B8E535C31360276D
:103F300014700BA22292E0B392E1440480D6147074
:103F40000BA22392E0B392E1440880C8147008A247
:103F50002492E0440C80BD74FC80B9E535147025D2
:103F60007408304D12304E04440680A8304F04448B
:103F70000380A14407809DA24E92E0A24F92E1A24D
:103F80001592E2808F1470117410A22292E0A22385
:103F900092E1A22492E2023F141470097418A21F45
:103FA00092E0023F14147015D2E3A26592E4A26677
:103FB00092E5A26792E6A26892E7023F14E4023F0C
:103FC00014E536B44106753404023EE2B44214E509
:103FD000356003301B05C21B12978F75591E744242
:103FE000023EDFB4440280F8B44B028003024089F1
:103FF000E53554F8B4083AE5355407700A741912D7
:1040000083DAE5360240C2B4010A74191283FBE573
:10401000360240C2B4020A741912841CE53602400A
:10402000C2B4030A741912843DE5360240C2023E4E
:10403000B3B42003023EB3B4282BE53520E00830AA
:10404000380B1254DD8006203803120C7AE535A2B5
:10405000E09238757A1F7561015003756102E5368B
:10406000D24C023EDFB4300CE53554F8127E69E5DF
:1040700036023EDFB4380CE53554F8127E95E5364D
:10408000023EDF023EB3023EB3B4430FB5350375C3
:1040900044057534077535B0023EE2B44A2AE53569
:1040A0007023204F20204D0A741912701AC2141266
:1040B0006FCDC2AF75181075190F751AF0129723CE
:1040C000E536023EDF023EB3B44506753406023ED5
:1040D000E2B4510675340C023EE2B44D0EE53512E1
:1040E0008266E5365002B2E7023FE0B4490FE8C00D
:1040F000E078C1E535F2D0E0F8744980C5B44C06EB
:1041000075340E023EE2B4460280B7B4470280B274
:10411000B44848E8C0E0D25DE535B40004D25E8022
:1041200032B4011F78BCE2602A78BEF2C25B741917
:10413000543F4480C2AF7518C0751909F51A12971B
:10414000238010B40207121281600880DFD0E0F8EB
:10415000023EB3D0E0F874480240C2B44F08129651
:10416000F3744F0240C2B45917E5357029E8C0E036
:1041700078B6E2F535D0E0F8745975340D023EE2B8
:10418000B45A13E8C0E0789DE2F535D0E0F8745AEF
:10419000753405023EE2023EB3E565B4000122C279
:1041A000AC129671129671D299E565B40706124366
:1041B000AD02420BB401061210EA02420BB4030630
:1041C00012117702420BB40206120FFB02420BB42B
:1041D000040612104502420BB405061203090242FE
:1041E0000BB406061211C702420BB40906126EDEAA
:1041F00002420BB40E06126F6202420BB41006129A
:1042000044AF02420BB411030256A0C241D2B6120F
:10421000724575650022E565B4000122B411030200
:1042200056A0B40203120FF2C241D2B61272457503
:10423000650022D3223012FBE570540260F578103D
:10424000E2F58308E2F5822418E58334FC40E412A9
:104250005CE47812E2B4180040D97401F9747BF878
:10426000752F007530007531001205397401F9742D
:104270007CF8752F017530F87531FF120539125C25
:10428000F2122486257BF57B7824E2FAC3E57B9A3B
:10429000F57B125CF27824E21224AC125CF2124F2D
:1042A000747885E2257CF57C7923E3F2FAC3E57C1A
:1042B0009AF57C125CF2124F97125CF2E58275F06F
:1042C00008A42420F582500205F0A8F0E58375F0DB
:1042D00008A4282400F5837408F9748CF8752F005D
:1042E000858330858231120539788CE57B7A082602
:1042F00008DAFCF57B789C79137A0A75F00FE354A1
:104300000FF652F00809DAF643F0F0E5F004126512
:104310009D78A8791D7A0675F00FE3540FF652F0D8
:104320000809DAF643F0F0E5F0041265A57408F91F
:10433000748CF8752F008583308582311204C6781D
:104340008CE57B7A08C39608DAFBF57B125CF212E7
:104350004E3CC082C08378007A06E2257CF57C085A
:10436000DAF8D083D0827406F97425F8752F0185A8
:10437000833085823112049579257A06E3C57CC3A2
:10438000957CF57C09DAF57401F9747BF8752F00DA
:104390007530007531001204C67401F9747CF8752B
:1043A0002F017530F87531FF1204C6C32212698FD0
:1043B000C2B67537007403125608E51E125608E59A
:1043C0001F1256087450125608747D125608900039
:1043D00000E535600F9003E81460099007D0146081
:1043E00003900BB87E7D7F0875F000C0F012698FD6
:1043F000B40203D38001C3D0E033F5F0A3DFEC12A5
:104400005608DEE2E53712560874FF125608309956
:10441000FD12965922023DA28599F0543F60F6B4F0
:104420000108E5F0B51E32023BE1B40208E5F0B543
:104430001F27023BE1B40307E5F0F540023BE1B47E
:10444000041AE5F0F541600BB44000500C753F458F
:10445000023BE1753F44023BE1023D7EB40516E5B7
:10446000F0B542F5754320753F0012724DC241759B
:104470006510023BE724FAB42000500AC0E0241083
:10448000F8E5F0F2D0E005E0B54104E5F080C4E5E0
:10449000F0023BE18540367535000244ABE540440F
:1044A00080F53675350174017810F21245B122E5B8
:1044B00040B42845E54124FD50E3C082C083781014
:1044C000E2F58308E2F58208E2B4030A7419125493
:1044D000E91268BD801DB4020A74191255181268D9
:1044E000678010B4010A741912552112689D800367
:1044F0001268A1D083D082809BB42927E54124FE95
:1045000040028099C082C0837810E2F58308E2F50A
:104510008212698F7812F2753503854036D083D0C8
:10452000828088B42A21C082C0831267E87419543B
:104530003F4400C2AF7518C075190BF51A129723C6
:10454000D083D082024494B42F1DC082C083124510
:10455000F27810E583F208E582F27535028540367F
:10456000D083D0820244ABB43013C082C0831242E5
:1045700035D083D082400302449402449DB4330E6C
:10458000C082C083124591D083D0820244AB0244E2
:10459000AE7537007403125608E51E125608E51F63
:1045A000125608743312560874201256081263E625
:1045B00022C2B67537007423125608E51E1256083B
:1045C000E51F125608E536125608E535125608E57D
:1045D00035600E7810E2F5F0E5F012560808D53592
:1045E000F4E53712560874FF1256083099FD1296FA
:1045F0005922D2B675F001129625D5F0FAE51DD2F2
:1046000075B51DFD2421900000A2B092D5A2D53031
:10461000B001B35003B2D5A3B51DF2C27575F00158
:10462000129625D5F0FA22E55AC2546002D2547887
:1046300099E54FF2788076FFC264C23A20440C209C
:10464000421B304303024769024D24120101787F67
:10465000E2F58308E2F582121E220247D61201011A
:10466000122063121E976019121F2D603D1233F83D
:10467000C2AF75182075190F751AEC1297230246F0
:10468000AD12557EB40206124C6E024D24B4031ACC
:10469000C082C0831200E3122E04D083D082304344
:1046A0000CE53B6008121DB370030247D6754796B0
:1046B000D54419C2AF7518C0751900751A531297F1
:1046C000237544057571007406127E69126E6502C9
:1046D0004D127562051233F8C2AF7518C075190016
:1046E000751A07129723754E041233E11233F775CA
:1046F000F06412011D024D24205024E56C54086022
:10470000CB301218C0E0C082C0837411120189D06E
:1047100083D082D0E0400280B9024740024740E5A2
:104720006B548060A7301218C0E0C082C083741040
:10473000120189D083D082D0E040028095024740A8
:10474000128542401E204F15302903203809900F52
:10475000E9124D6A024D24124C98024D24124CA4C9
:10476000024D24124CAA024D24E53B608B78A8E64A
:10477000B40A030254CF121FC2703912557EB4011D
:1047800006124C6E024D24B403241200E3C082C012
:1047900083122FF7D083D082304216C082C083129A
:1047A0000101122063D083D082121CC07003024723
:1047B000D60246AD1255B040131233F8C2AF751889
:1047C0002075190F751AEB12972380E51250EBC272
:1047D00043D24202466030502D301219C0E0C082F0
:1047E000C083740C120189D083D082D0E0400302D0
:1047F00048060247F57567027896E27898F21251FA
:10480000F250030246AD30512D301219C0E0C08283
:10481000C083740D120189D083D082D0E04003029E
:1048200048360248257567037897E27898F2125166
:10483000F250030246AD12746C4008C289C28BD29A
:10484000B4C2947887E2047011C2AF7518208583D2
:104850001985821A1297230246AD754700754405E3
:10486000E570540170057407127E957406127E95EA
:10487000203A057405127E95C082C083124ED6D0B0
:1048800083D0825006124CBF024D24E58224CEE52F
:104890008334FF5056124E2A4051E56D5480700308
:1048A000024B80C2A1D24AD2A4C249754E00123333
:1048B000E11233F7121E22C082C083024AF5124C65
:1048C000AA024AA6124CA4024AA6124C98024AA670
:1048D000124E33500F124FB630E109302929124CD5
:1048E00098024D24D264C25D024B80A25030360142
:1048F000B3921012854240C6204FC9303809E56D89
:10490000542070CC2029C33050037886E230510304
:104910007887E2120159500902495D124C92024A0D
:10492000A63012F73035F41253B4403130102E3027
:104930001218C0E0C082C0837409120189D083D0EC
:1049400082D0E0400280D402494AC082C08312690A
:10495000FAD083D0825006124CB0024AA6787F76F5
:10496000FFD231301219C0E0C082C083741412012A
:1049700089D083D082D0E0400302498102497FC2BE
:10498000311253B45003024A1430101C126A4F50B3
:104990001730310812698FB40202800C124C7A026F
:1049A0004AA6124C9E024AA61255CE40F512698FB5
:1049B000B4000520102A8046B4013D201022301C8E
:1049C00053757710C2AF7518C0751900751A0912A2
:1049D0009723203106124CB5024AA6124DF38034BB
:1049E000E56D5410700912553378807602802512D7
:1049F0005533787F7602801CB402DA2010C0E56D52
:104A0000541070091255337880760180071255339F
:104A1000787F7601C082C083120705D083D0825090
:104A200006124CBA024D2430125C1253B440573077
:104A30001219C0E0C082C0837408120189D083D0EB
:104A400082D0E04003024A86024A4B20541CA25006
:104A500092537881A6837882A682124DEFC250C20B
:104A6000511200F7755A02024D24755A00E58378F9
:104A70008166F5F0E58278826645F07006124CC4D6
:104A8000024AA612545A124D6AE56D54106006305F
:104A9000160312553EE56A5410600BC082C08312A3
:104AA0004FEFD083D082E56D5420600C30640975DF
:104AB000F0C812011D024D24124E335009124FB698
:104AC00030E103024D24C2A1D24AD2A4C249754E9C
:104AD000001233E11233F7121E22C082C083E56D4B
:104AE00054807006122FF7024B3D122FF130424DC9
:104AF000121CC070481200E375F06412011D122FE1
:104B0000F1304239121CC070341200E375F06412A7
:104B1000011D122FF1304225121CC070201200E33B
:104B200075F06412011D122FF1304211121CC07079
:104B30000C1200E375F06412011D122FF1D083D026
:104B40008220440920421720431F024D24120101F4
:104B5000787FE2B5830D08E2B58208024B80121C13
:104B6000C0601D126E65024D12E53B60F6121DB36A
:104B7000600E1255B050EC1250EBC243D24280DEB0
:104B8000788076FF301219C0E0C082C083740612AC
:104B90000189D083D082D0E04003024BC0024BA0F9
:104BA000E56A54016026E582458360203050037831
:104BB00086E23051037887E21201595009024BCC4A
:104BC000124C80024D12124C80024D24A238926386
:104BD000128550500F124C8675F01E12011D1200E6
:104BE000C0024D24128562500F124C8C75F01E12BB
:104BF000011D1200C0024D24B238757A1FD26D1209
:104C000033F8303825C2AF75187085831985821A3C
:104C1000129723125594757303C2A3C248D2A1C23E
:104C20004AD2A4C249120C7A803EC2AF7518608580
:104C3000831985821A1297231212AF1255A3757326
:104C400003D2A3C248D2A1C24AC2A4C2491254DDAF
:104C5000E56D54206012E58224CEE58334FF5005D3
:104C6000124E2A50030249071200D6024D24126E3A
:104C700065024CC7126E65024CC7126E65024CC7C6
:104C8000126E65024CC7126E65024CC7126E650249
:104C90004CC7126E65024CC7126E65024CC7126E8D
:104CA00065024CC7126E65024CC7126E65024CC796
:104CB000126E658012126E65800D126E658008128C
:104CC0006E658003126E65755A00788176FF788272
:104CD00076FFD2611233F8C2AF751820858319852B
:104CE000821A1297231200C0C26122E56B54087029
:104CF0000320501DE54F04601814F5F0788BE26531
:104D0000F0600EC2AF7518C0751901854F1A129761
:104D10002322D2611200AAC261755A00788176FFFF
:104D2000788276FFC243C2427899E2F54F7880E6F6
:104D3000B4020A741C125518126867800BB401087B
:104D4000741C12552112689D788076FFE56D5480A1
:104D50006017306D1475F0FF12011D75F0FF120120
:104D60001D75F0FF12011DC26D22D27230380EC2C5
:104D7000A3C248C2A2C24BD2A4C249800CD2A3C2D1
:104D800048C2A2C24BC2A4C249A2509214D213126A
:104D90006E65741C12701A126FCDE56A544060067D
:104DA00020A80312932F1233F8124CEBC2AF7518E0
:104DB0001085831985821A129723E56E540860299D
:104DC00012128160241233F8C2AF7518E08583197E
:104DD00085821A129723741C543F4480C2AF751801
:104DE000C0751909F51A1297231200D6C272221241
:104DF0006E6522126E65227408F9748CF8752F01A5
:104E00007530007531001205397891E6085608565C
:104E10000460141200E3122E04304309E53B6005E0
:104E2000121DB36002C322D32222E582249CE583B3
:104E300034FF22E582249CE58334FF22E58275F06D
:104E400006A4F582A8F0E58375F006A428F583E5AD
:104E5000822400F582E5833465F583C082C08374C3
:104E600006F97400F8752F01858330858231C0F012
:104E70001204F7D0F0D083D082227892E630E40298
:104E8000240A2323543CF5837891E6C4540375F037
:104E90000AA4F5F0E6540F25F0030303F5F053F0F0
:104EA000E085F08254034583F5837890E6C454038B
:104EB00075F00AA4F5F0E6540F25F04582F58278E6
:104EC00093E6547F788CF608A68308A68222C3EC6A
:104ED0009FEB9EEA9D221253B45003024F2A124EBA
:104EE0003C7800E2B4FF03024F2A127896124E7A01
:104EF000788CE6FA08E6543FFB08E6FC7800E2FD11
:104F000008E2543FFE08E2FF124ECE401F788CE6C6
:104F1000FA08E6543FFB08E6FC7803E2FD08E25499
:104F20003FFE08E2FF124ECE5002C322D3221224CB
:104F300086C0E02400F582E434D3F5837401F9746B
:104F400086F8752F01858330858231C0F01204F711
:104F5000D0F0D0E02400F582E434D4F5837401F974
:104F60007487F8752F01858330858231C0F0120473
:104F7000F7D0F022E5822400F582E58334C3F5837F
:104F80007401F97485F8752F01858330858231C0ED
:104F9000F01204F7D0F022E5822400F582E5833494
:104FA000C3F5837401F97485F8752F018583308505
:104FB00082311204952230122BC082C083124F74AA
:104FC000D083D082C082C083124F2ED083D082E59E
:104FD000822418E58334FC40077885E24402F222FB
:104FE0007885E222E47886F27887F27885F22212D8
:104FF000248660432323C0E05403F5F0D0E054FC42
:105000002400F582E5F034D5F5837404F9748CF846
:10501000752F01858330858231120539788C799E10
:1050200075F004E6F30809D5F0F975F0031296253A
:10503000D5F0FA1234A02274FF789EF208F208F23A
:1050400008F280E6786BE2540FC4F58308E2540F4F
:10505000428308E2540FC4F58208E2540F4282E50D
:10506000822460E58334F022786575F006E2540FFF
:1050700008D5F0F9E2540F75F00AA4F582758300A3
:1050800008E2540F2582F582E58275F00AA4F582C4
:1050900085F08308E22582F58250020583E582755A
:1050A000F00AA4F582C0F0E58375F00AA4D0F025DB
:1050B000F0F58308E22582F58250020583E582241B
:1050C00060E58334F022D3227865E2600BF5F008C6
:1050D000E224F64005D5F0F7C322D3227865799C07
:1050E00075F00AE2F70809D5F0F922C082C083788A
:1050F0009C9001F075F00AE0F608A3D5F0F9900154
:10510000FAE0F564D083D08222C082C083789C907C
:1051100001F075F00AE6F008A3D5F0F9E564900116
:10512000FAF0D083D082221250DC121CC022D0832D
:10513000D082221250DC125109122E76C082C08316
:10514000753B0175F0057865E2540F70E108D5F004
:10515000F7E208540FF9E208540FC4F5F0E20854DE
:105160000F45F0FAE208540FC4F5F0E208540F4579
:10517000F0FB12943AEC70B678A8C258EDC4125104
:10518000A3ED1251A3EEC41251A3EE1251A3EFC42A
:105190001251A3D258EF1251A3E82458F53BD08303
:1051A000D08222540F7003305804D258F608227966
:1051B000A877000975F00577FF09D5F0FA2212509B
:1051C000DC1251091251AF75F0087867753B06E2A1
:1051D000540F700608D5F0F7800979A8E2F708099E
:1051E000D5F0F9221251BE121DB322125133121DF5
:1051F000B322C082C0837898E270030252B724FDC4
:10520000403C1200E312536E20441920430B3042FD
:1052100010121CC0700B0252B7121DB37003025261
:10522000B70252B4D083D082C082C083787FE2B507
:1052300083EF08E2B582EA658270E60252B7E224A3
:10524000E250691200E3127C6B5006D083D082D307
:10525000227898E275F00384E5F0B4000A1253C294
:10526000121DB370E6803DB4011B7898E2B42203AE
:10527000206C0A1253F3121CC070D08027127CA439
:1052800050DE022DFFB402221253F640BEE58285A5
:1052900083F0D083D082C082C083658270ADE5F098
:1052A000658370A7D083D082C322809F1200E3124F
:1052B0007C195009025368D083D082C3227898E2C7
:1052C000B40F11127C0640EC1251E460EA1251272F
:1052D00060E580E0B4100C127C0640D81251EB60FF
:1052E000D680EAB4110B127C0640C9125044025316
:1052F0001AB4030C127C0640BB1251E470B680B79E
:10530000B4040C127C0640AC12512770A780A8B4DC
:105310000523127C06409D1250684098E5828583E3
:10532000F0D083D082C082C08365827087E5F0654B
:105330008370818082B41205127C12808BB41305B5
:10534000127C128097B41705127C12809EB414B0A0
:10535000127C1280A4B415B7127C1280ABB416056F
:10536000127C1280B20252B4D083D082D32275460E
:1053700032D24C304609C246C067120273D067E58C
:1053800046D36018C244C243C242122C8050E41279
:10539000362B2044062043033042D8C3C0D0A86730
:1053A0007405B802027404D0D040051235DC8003C5
:1053B00012360422E582B4E807E583B40F02D32253
:1053C000C3221250C85002D3227865E260F9B409B2
:1053D000047408800250FAF5F008753B06E2540F99
:1053E000700608D5F0F7800979A8E2F70809D5F02A
:1053F000F9C322027DFD1250C85004D322C3227883
:1054000065E20860F6B40108E2F58275830080ED7C
:10541000B40212E275F00AA4F58208E22582F58250
:1054200075830080D8B40320E275F00AA4F58208E1
:10543000E2258275F00AA4F58285F08308E22582D0
:10544000F58250B9058380B5B404057866025074BE
:10545000C39404F5F0786602506DB250B251754EA7
:10546000071233E11233F7B251B250C2AF7518C010
:10547000751900751A0C12972330530EC2AF7518A8
:10548000B0751900751A00129723124CEBC082C038
:10549000837881868378828682C2AF75181085836F
:1054A0001985821A129723D083D08222E53BB40358
:1054B0001C78A8E6B40A1608E624F6401008E6248C
:1054C000F6400A18E675F00AA40826C322D3221271
:1054D00054AC500302477678B9F20225E6120C7AF2
:1054E0001296F31296FDC23A22301C2B543F44C050
:1054F000C082C083C0E0C2AF7518E0858319858281
:105500001A129723D0E0C2AFF51A75190E7518C09C
:10551000129723D083D08222301CFC543F448080D9
:10552000CF301CF3543F444080C6301CEA543F4403
:105530000080BD78B7E582F278B8E583F222787F03
:10554000E6B40118C082C08378B7E2F58278B8E289
:10555000F583741C12552112689D8019B4021AC07B
:1055600082C08378B7E2F58278B8E2F583741C12C2
:105570005518126867D083D082787F76FF22E420A6
:105580005009A26592E0A26692E122A26792E0A28F
:105590006892E122E56E54016008304E05741D12D8
:1055A00083DA22E56E54016006787EE66460F622B6
:1055B00078942051027895E2B40F02D322B41002FD
:1055C000D322B41202D322B41302D322C32278C14D
:1055D000E2B4010520100FD322B402053010078079
:1055E000F6B4030280F1C322C5372537C53722E55B
:1055F0004724F34008D2A3C248D2A2C24B3098EF4E
:10560000C298E5991255E8223099FDC299F5991290
:1056100055E822C2A3C248C2A2C24BC2B675370027
:105620007405125608E51E125608E51F1256082288
:10563000129671129671129671125613E536125621
:1056400008E53712560874FF1256083099FD129675
:10565000592212093402565B1208D0C0E0125613C8
:10566000E536125608D0E0125608E537125608748F
:10567000FF1256083099FD12965922129671125651
:1056800013E5361256087900E312560809DDF9E5EC
:105690003712560874FF1256083099FD1296592297
:1056A000C28EC28CC2ADC2ABC2ACC2AF7581B59066
:1056B00056BAC082C08375D00032D2AFD28C127974
:1056C000BB1215A71215DBD21D75470F751A0012F4
:1056D00096F3E538600854F87004C206D26AE539DA
:1056E000600854F87004C207D26AE53A600654F8BC
:1056F0007002C20812701312724DD29912563012F3
:10570000970D75470FD29802570AD2B6D2A3C24856
:10571000D2A2C24B1255EFB40AF0F5371255EFB5CD
:105720001EF51255EFB51FEF1255EFF536B46D03A8
:105730000257CCB46E030257EBB46F03025826B481
:105740007003025873B47103025887B4730302588C
:1057500098B474030258B8B475030258CCB47703F4
:105760000258E4B478030258F8B4790302591DB41E
:105770007A03025939B46C0302594DB46B030259D0
:105780006FB46A030259B2B469030259B4B468032E
:10579000025A1BB46703025A33B46603025A4EB46A
:1057A0006503025A6DB463030260AEB46103026123
:1057B00024B4310302616EB432030261B3B4330323
:1057C000026321B4340302637302570AAF371255E0
:1057D000EF6F70F5125630125630125630D2B67541
:1057E000F01E129625D5F0FA0274671255EFFD14DB
:1057F00024E0402F1255EF2400FC7B001255EFFEF1
:10580000AF371255EF6F701B8EF0EDF97400F88B07
:105810002F8C3085F031C0F01204F7D0F012567B97
:1058200075470F02570A1255EFFD1424E040F41299
:1058300055EF2400FC247140EA7B021255EFFEED87
:10584000FA78001255EFF208DAF9AF371255EF6F18
:1058500070D1C2A3C248C2A2C24B8EF0EDF974004F
:10586000F88B2F8C3085F03112049512563975471C
:105870000F80B0AF371255EF6F70A81208001256A4
:105880003075470F02570AAF371255EF6F70261267
:10589000565875470F02570A1255EF1255EF125519
:1058A000EFAF371255EF6F700C1267E81256307574
:1058B000470F02570A0258231255EFFD1424E04007
:1058C000341255EF2400FC7B010257FC1255EFFD0A
:1058D0001424E040201255EF2400FC240640167BDF
:1058E0000302583BAF371255EF6F700912565275CD
:1058F000470F02570A02582379507D071255EFF3DC
:1059000009DDFCAF371255EF6F70EA78937600121D
:105910006A6F40E112783212563902570AAF3712D5
:1059200055EF6F70D0127896129671125613E536B5
:1059300012560812032502570AAF371255EF6F703F
:105940006E120D9412563075470F02570A1255EF1A
:10595000FE1255EFFD1255EFFCAF371255EF6F7089
:105960004E12076F404912563075470F02570A1200
:1059700055EFFE1255EFFDAF371255EF6F70301235
:10598000074E129671129671125613E5361256088A
:10599000EE125608ED125608EC125608E53712566C
:1059A0000874FF1256083099FD12965902570A02E0
:1059B000582380FBAF371255EF6F70F31208C860A1
:1059C000027401C0E012092C60027402D0F045F0AC
:1059D000700A1208171219561215AEE4C0E01256DA
:1059E00013E536125608D0E0C0E0125608E537122B
:1059F000560875F003129625D5F0FA125613E536BF
:105A0000125608D0E0125608E53712560874FF12F5
:105A100056083099FD12965902570A1255EFFD1497
:105A200024E040271255EF2400FC2471401D7B0028
:105A300002583B1255EFFD1424E0400F1255EF249D
:105A400000FC240640057B0102583B025823AF3777
:105A50001255EF6F70F5129671129671125613E58A
:105A6000361256081263E602570A0258231255EFFF
:105A7000F5831255EFF5822460E58334F040EB1294
:105A80005CE41255EFFDB41B0040DF1424E040DA63
:105A9000780075F02074FFF208D5F0FB78001255FD
:105AA000EFF208DDF9AF371255EF6F70BDE57054B6
:105AB00002600D125CF2E5822418E58334FC40AAF2
:105AC00012563075F005129625D5F0FA1256397532
:105AD0001A01301295E57054027070125D1A125D51
:105AE00000125CF2121E22789C79007A0A75F00F7F
:105AF000E3540FF652F00809DAF643F0F0E5F0044B
:105B000078A579907428121CCF600B125BA95006FF
:105B1000751A03025A6A125D00125CF2121E227894
:105B2000A8790A7A0675F00FE3540FF652F00809C7
:105B3000DAF643F0F0E5F00478AD79937418121CAE
:105B4000CF6008125C3E5003025A6A125D00125D7B
:105B50002A751A6502570AC0E07865E583F208E500
:105B600082F2D0E022C0E07867E583F208E582F2B5
:105B7000D0E022C0E07865E2F58308E2F582D0E06B
:105B800022C0E07867E2F58308E2F582D0E022E502
:105B9000822400F582E5833425F58322E582240002
:105BA000F582E5833445F58322125CF2AB83AC8247
:105BB0007530257900752F03C03075310090008C49
:105BC00012043A1205C912043A12061390008C7A94
:105BD00080E0A3F5F0E0A36C7005E5F06B6012DAED
:105BE000F0D0300530E53034BA50C87405F51AD31A
:105BF00022D083EA2AF5F0E4C395F0F582125B57D0
:105C0000789C79007A0A75F00FE3540FF652F00889
:105C100009DAF643F0F0E5F004600B121E89700912
:105C20007406F51AD322121E89E5822582F582E5D3
:105C3000833583F583125B8F125B65025EB4125C61
:105C4000F2AB83AC827530457900752F03C0307597
:105C5000310090008C12043A1205C912043A12065F
:105C60001390008C7A80E0A3F5F0E0A36C7005E55A
:105C7000F06B6012DAF0D0300530E530349A50C85D
:105C80007407F51AD322D083EA2AF5F0E4C395F01D
:105C9000F582125B5778A8790A7A0675F00FE354FB
:105CA0000FF652F00809DAF643F0F0E5F004601C54
:105CB000121FB4701AAB83AC82125CF2EBB5830690
:105CC000ECB58202C3227404F51AD322121FB4E584
:105CD000822582F582E5833583F583125B9C125B16
:105CE00065025EB4C0E07869E583F208E582F2D02F
:105CF000E022C0E07869E2F58308E2F582D0E02294
:105D00007400125608740012560874001256087473
:105D1000001256087400125608227F017E257583F2
:105D20000375822574401207C1227401F9747BF84F
:105D3000752F007530007531001205397401F97442
:105D40007CF8752F017530F87531FF12053978161A
:105D5000E20470067811E204601D125CF2122486DF
:105D6000257BF57B7811E2FAC3E57B9AF57B125C23
:105D7000F27811E21224AC125CF2124F747885E2D0
:105D8000257CF57C791AE3F2FAC3E57C9AF57C125E
:105D90005CF2124F97125CF2E58275F008A42420A1
:105DA000F582500205F0A8F0E58375F008A42824D8
:105DB00000F5837408F9748CF8752F00858330859D
:105DC0008231120539788CE57B7A082608DAFCF5F1
:105DD0007B789C79007A0A75F00FE3540FF652F045
:105DE0000809DAF643F0F0E5F00412659D78A87929
:105DF0000A7A0675F00FE3540FF652F00809DAF646
:105E000043F0F0E5F0041265A57408F9748CF87598
:105E10002F008583308582311204C6788CE57B7A29
:105E200008C39608DAFBF57B125CF2124E3CC08286
:105E3000C08378007A06E2257CF57C08DAF87800E1
:105E40007918E3F2087912E309F208E3F208791904
:105E5000E3F2087914E309F208E3F2D083D0827404
:105E600006F97400F8752F0185833085823112049C
:105E70009579007A06E3C57CC3957CF57C09DAF553
:105E80007401F9747BF8752F0075300075310012BC
:105E900004C67401F9747CF8752F017530F87531FA
:105EA000FF1204C67F037E25758301758225744029
:105EB0001207C122125B81E5828583F0125B73C3F6
:105EC0009582C0E0E5F09583D0F045F07002C322E2
:105ED0005003025FD0125B81C0E0C3E58224FEF56F
:105EE00082E58334FFF583D0E0125B65E58285832C
:105EF000F0125B73B58207E5F0B58302C322125B33
:105F000073AF83125B81EFB58310AE829000697826
:105F10008CE0F6A308E0F6025F327EFE8F830583F5
:105F20007402F9748CF8752F038583307531001273
:105F300005397900752F038F3075310090008C1270
:105F4000043A1205C912043A1206138F83758200AF
:105F5000125B737D00E5836F7002AD82ED248CF5DA
:105F60008275830050020583C3EE9D20E05C03FC34
:105F70006017C082C083A3A3E0FAA3E0FBD083D064
:105F800082EAF0A3EBF0A3DCE9EE248CF5827583C2
:105F90000050020583788CE6F0A308E6F0790075DE
:105FA0002F038F3075310090008C12043A12065383
:105FB00012043A120667852F32853033125B81EF67
:105FC000B583030260A60F025F037408F51AD3229B
:105FD000125B73AF83125B81EFB58310AE829000CA
:105FE00069788CE0F6A308E0F60260047E008F83F7
:105FF00015837402F9748CF8752F0385833075311D
:10600000FE1205397900752F038F3075310090002D
:106010008C12043A1205C912043A120613125B7369
:106020007DFEE5836F7002AD82ED248CF582758371
:106030000050020583C3ED9E20E06D03FC6026C086
:10604000E0C3E58224FEF582E58334FFF583D0E0EA
:10605000C082C083E0FAA3E0FBA3EAF0A3EBF0D098
:1060600083D082DCDAEE248CF58275830050020541
:1060700083788CE6F0A308E6F07900752F038F3063
:1060800075310090008C12043A12065312043A1231
:106090000667852F32853033125B81EFB5830302AB
:1060A00060A61F025FD5C3227409F51AD3221255C8
:1060B000EFF5831255EFF5821255EF700D1255EF83
:1060C0007008AF371255EF6F6009025823D01FD008
:1060D0001E80F7C01EC01F12252E40F185831E852D
:1060E000821F121C9A1279BB7401F9748CF8752FF7
:1060F00000753000753100120539788CE6C3951EA5
:10610000C3951FD01FD01E251E251FF67401F974DC
:106110008CF8752F007530007531001204C61256C8
:106120003002570A1255EFF583AF371255EF6F70F3
:1061300099129671129671129671125613E53612D3
:106140005608E4125608E51A125608E4125608E4F6
:10615000125608E4125608E4125608E5371256089B
:1061600074FF1256083099FD12965902570A1255BB
:10617000EFFC24EF40211255EFFD1255EFF583128D
:1061800055EFF582788CECFB1255EFF608DBF9AF92
:10619000371255EF6F600302570A7547F0ECF97438
:1061A0008CF88D2F8583308582311204C6125630CB
:1061B00002570A1255EFFC24EF40161255EFFD125C
:1061C00055EFF5831255EFF582AF371255EF6F603B
:1061D0000302570A7547F0ECC0E0ECF9748CF88DB7
:1061E0002F8583308582311205391296711296718E
:1061F000129671125613E536125608D0E0FC788CD0
:10620000E612560808DCF9E53712560874FF1256F4
:10621000083099FD12965902570A85832F858230DE
:1062200075310012043A1205C9752F037530FA75DD
:10623000310012043A1206677532FF7533FF22C02F
:1062400082C083752F037530FA75310012043A123B
:1062500005C9D083D08285832F85823075310012A5
:10626000043A1206677532FF7533FF227455788C35
:106270007910F608D9FC7410F9748CF885832F8591
:1062800082307531001204C67532FF7533FF741009
:10629000F9748CF885832F858230753100120539A9
:1062A000788C7910B6553B76AA08D9F87410F97431
:1062B0008CF885832F8582307531001204C67532C3
:1062C000FF7533FF7410F9748CF885832F85823045
:1062D000753100120539788C7910B6AA0508D9FAFB
:1062E000E422740122E5822400E58334F8402CC0C6
:1062F00082C08312621AD083D082C082C0831262AD
:106300006CD083D082C082C083C0E012623FD0E0F4
:10631000D083D0827007A3DECCE422740B22025813
:10632000231255EFFE1255EFF5831255EFF582AFAC
:10633000371255EF6F70E775470F1262E5C0E01234
:106340005613E53612560874081256087400125691
:1063500008E583125608E582125608D0E012560866
:10636000E53712560874FF1256083099FD129659F7
:1063700002570A1255EFF5831255EFF582AF371227
:1063800055EF6F709912967112967112967112569E
:1063900013E536125608E583125608E582125608B0
:1063A000E53712560874FF1256083099FD129659B7
:1063B000129671129671129671125613E536125694
:1063C00008E583125608E582125608E5371256088A
:1063D00074FF1256083099FD129659E58312726EB9
:1063E00075470F02570A7406125608744D12560864
:1063F0007403125608740312560874061256087471
:1064000004125608748D125608742012560874F936
:106410001256087400125608740F12560874A0120F
:10642000560874801256087400125608740F1256DB
:106430000874A012560875F000200108300210758B
:10644000F050800B20020575F057800375F041E590
:10645000F0125608740212560812252EE433125612
:106460000874001256087400125608740012560878
:1064700074001256087400125608740012560874FC
:106480000012560874001256087400125608740060
:10649000125608740012560874001256087400123E
:1064A0005608E53712560874FF1256083099FD1247
:1064B0009659229064BBC082C083327581B575D075
:1064C000000274671208D0C0E07401F9748CF8758A
:1064D0002F00753000753100120539788CE6D0F048
:1064E000C395F0F67401F9748CF8752F00753000BF
:1064F0007531001204C622788C75F00876FF08D535
:10650000F0FAE47887F27886F22275F005C0F0128E
:106510002FF7D0F0204206204303D5F0F022751E5D
:1065200030751F3012252E1264F7C250C251D2A30B
:10653000C248C2A2D24BD2A1C24AD2A4C2491200BE
:10654000E312650A20420620430902659512659D03
:106550000265901265BD403D1200D612252E4030D6
:10656000122FED2042FA30392C1213BCB40B030267
:106570006590B40A00501E2430F51E122FED204203
:10658000FA3039111213BCB40A0050092430F51F37
:106590001200D6C32212252E1200AAD322789C798B
:1065A0008C7A05800678A879917A03E608540FC49E
:1065B000F5F0E608540F45F0F709DAEF22204229FA
:1065C000304326E53B600624FD24FC401C1265A5F3
:1065D0001200E3122FED20420B30390D1213BCB420
:1065E0000B07800312659DC322D3227401F97489BD
:1065F000F8752F007530CE753101C0F01204F7D058
:10660000F07889E2540F227401F9748AF8752F002A
:106610007530CE753100C0F01204F7D0F0798AE3FE
:1066200022788974FFF27401F97489F8752F007566
:1066300030CE753101120495798A74FFF27401F934
:10664000748AF8752F007530CE75310012049522CA
:106650000267351265EB60F8126607C0E09001EE44
:10666000748EF0A37400F0D0E0B4F0087889E230C2
:10667000E058C322B4E1129001EE749EF0A37400BE
:10668000F07889E230E143C322B4D2129001EE7473
:10669000AEF0A37400F07889E230E22EC322B4C3D6
:1066A000129001EE74BEF0A37400F07889E230E33A
:1066B00019C322798A74F0F37401F9748AF8752F7A
:1066C000007530CE753100120495D322B4F00374F6
:1066D0008E22B4E103749E22B4D20374AE22B4C3FA
:1066E0000374BE220266FE1266CC7F00FE788AE248
:1066F0001266CC758300F58274101207C122C21D88
:106700007548FA12421675F050129625D5F0FA1215
:10671000700C75F064129625D5F0FA12701375F0AE
:1067200014129625D5F0FA12008D75F06412962594
:10673000D5F0FA80C9C2AF7518C0751900751A5E18
:1067400012972375F0C8129625D5F0FA126D2F8096
:10675000AD798AF37401F9748AF8752F007530CE1B
:106760007531001204951266534093221266071287
:1067700065EB60C17889798AE3B4F008E230E1081A
:1067800074E180CDE3B4E108E230E20874D280C164
:10679000E3B4D208E230E30874C380B5E3B4C308BD
:1067A000E230E0D874F080A974FFF380F3B48E0374
:1067B00074FE22B49E0374FD22B4AE0374FB22B4B3
:1067C000BE0374F7220266FE1267ADC0E01265EBED
:1067D000D0F055F0F27401F97489F8752F00753016
:1067E000CE75310112049522756800756900126733
:1067F0006C9001EEE0F5821267AD758300C082C037
:10680000837410120799D083D08274101209B64095
:1068100001229001EEE01267C880CDC082C0839053
:1068200001EEE0F5F01267ADA3E0D083D0822582BF
:10683000C0E0E58335F0F8D0E0C322C082C08374A5
:1068400001F9748CF8752F0085833085823112052B
:1068500039788CB67A0CE56924FFF569E56834FF70
:10686000F568D083D0822212681BC082C083F58273
:1068700088837401F9748CF8752F008583308582C4
:1068800031120539788CB67A05D083D08222E56939
:106890002401F56950020568747A0268F5747980FC
:1068A0001EE5825583B4FF0CC082C0831267E8D016
:1068B00083D08222741912552A74788002747BFA6C
:1068C00012681BC082C083F5828883EAC0E074012D
:1068D000F9748CF8752F0085833085823112053963
:1068E000D0E0C0E0788C667007D0E0D083D0822200
:1068F00012683BD0E0C0E0788CF67401F97494F82B
:10690000752F007530CE7531021205397401F97496
:106910008CF8752F008583308582311204C674018E
:10692000F9748CF8752F0085833085823112053912
:106930007894E664646010D0E0C0E0788C66701DE6
:10694000D0E0D083D08222789476FF7401F97494D9
:10695000F8752F007530CE7531021204C69001EE25
:10696000E01267C8126607C0E0C068C0691267E835
:10697000D068D069D0E01266E7D0E0D083D082C082
:1069800082C083FA12681BF5828883EA0268F512D6
:10699000681BC082C083F58288837401F9748CF807
:1069A000752F00858330858231120539788CE6B4E5
:1069B00079077401D083D08222B47A077402D0831D
:1069C000D08222B47B077403D083D082227400D09B
:1069D00083D082221205A5C29374541205B0E4122A
:1069E000057F120592B47A04D293D322D9F4D293BC
:1069F000C3227532FF7533FFC3229001EEE0F583A9
:106A00001267AD75F00F752F00858330753100C0AA
:106A100083C0F012043A1205C912043A79001269CF
:106A2000D4D0F0D083058340C9D5F0DA752F008526
:106A3000833075310012043A1205C912043A79A064
:106A40001269D440AD7532FF7533FFD322C322E5FE
:106A500069456860F8789AE2F5F008E245F060ED83
:106A6000D3789BE2956918E2956822D0E0D322782A
:106A700055E254C070F7E275F00A84C445F0788E90
:106A8000F67854E254C070E5E275F00A84C445F02B
:106A9000788FF67853E254E070D3E275F00A84C43C
:106AA00045F07890F67852E260C354E070BFE2752A
:106AB000F00A84C445F0C0E07850E2030354C0D02B
:106AC000F045F07891F67851E260A254F0709EE2C1
:106AD00075F00A84C445F0C0E07856E254F8708B33
:106AE000E2C42354E0D0F045F07892F67850E2B456
:106AF00004005009F5F07893E654FC45F07893F6DD
:106B0000C32290050075F032C0F07402F9748CF85D
:106B1000752F01858330858231120539788DB6FF56
:106B200002801318E54F30120AB4FF0788F0788B03
:106B3000E2A8F0666011E5822414F5825002058314
:106B4000D0F0D5F0C3C322D0F0A3D32230124DE54C
:106B50008224FFF582E58334FFF58375F032E58208
:106B6000242CE58334F75005900500800AE5822443
:106B700014F58250020583C0F07402F9748CF87524
:106B80002F01858330858231120539788DB6FF0259
:106B9000800518E6B54F07D0F0D5F0C2C322D0F07B
:106BA000A3D32212011330120C126B024003900483
:106BB000ED126B4C22C04F126BD3D04F2230121308
:106BC000126B0240039004ED126B4C5005F54F120E
:106BD0006C0522E54F7005754F108023B4100575C4
:106BE0004F11801BB41105754F208013B42005751B
:106BF0004FFF800BB4FF05754F008003754FFF12E8
:106C00006D04E54F2222127896301A0FC21A126ACA
:106C10006F400512783280031278967891E6C4545A
:106C200003E6540F7892E6C45401E6540F7890E6D8
:106C3000C4540FE6540F788FE6C4540FE6540F2265
:106C400030120E126B025004126C0522126D048079
:106C5000FA80F8E56B5420700122E56E5402602A38
:106C600012798B502512250E5010C2AF7518C075C1
:106C70001900751A5A1297238016C2AF7518C0757D
:106C80001900751A5B129723800678B4E2D5E0727A
:106C900012789612724D129671129671D299C2B6EE
:106CA00074FF125608753700744212560874621247
:106CB00056087415125608742A125608741B125678
:106CC0000874001256087400125608740012560810
:106CD000740012560812033A75F010C0F0740012D6
:106CE0005608D0F0D5F0F4E53712560874FF125666
:106CF000083099FD129659C241D2B612724578B445
:106D000074FFF22222201C0122747512012E501CE5
:106D100020551BD2551267E8741A543F4400C2AF85
:106D20007518C075190BF51A12972322C25522C285
:106D3000AC129772600CF5188819120DF712978F24
:106D400080EFD2AC227E007F9C90000075F000E4C2
:106D50009325F0F5F0A3C3E5829EE5839F40F0E51F
:106D6000F0700122E583127074E582127074C2AD76
:106D7000C2ACD21DD2A3C248D2A2C24BC2A1C24A47
:106D8000D2A4C24980EE30123F740078B212013FA3
:106D900040367F087E00747812012ECE13CE05E0B7
:106DA000DFF6201E0F740078B312013F5006EE7814
:106DB0007D666014EE787DF6F54FC2AF75183075BC
:106DC0001901854F1A12972322C2AFF51A75190FB0
:106DD000751810029723223012FC204DF9740178A7
:106DE000B212013F40F0747712012EE492E0C0E04D
:106DF000747612012ED0E033FE201E0F740178B39A
:106E000012013F5006787EE66E60CBEE787EF6206B
:106E1000E10630E028026E5030E014A24F724E506E
:106E2000B5C24FC24E126FFD74F8126DC980A7D261
:106E30004FC24E126FFD74F7126DC98099204E0E2D
:106E4000D24EC24F126FFDD24C74F6126DC98086BD
:106E5000A215824E40F8D24EC24F126FB174F51295
:106E60006DC9026DD6C082C083D083D08222D2A3E6
:106E7000C248C2A4C249223038F4C2A3C248D2A434
:106E8000C2492220120122747312012EE492E0C042
:106E9000E0747412012ED0E092E1F5F0657453F0C5
:106EA0000385F074201E026009E5F00303441A1202
:106EB00093D1747112012EE492E0C0E07472120159
:106EC0002ED0E092E1F5F0657553F00385F0752062
:106ED0001E026009E5F00303441A1293E722C2B6CA
:106EE0007537007403125608E51E125608E51F1286
:106EF0005608744E12560874081256087401125639
:106F00000874061256087857E2F5F0E5F0125608B4
:106F100008E2F5F0E5F01256087859E2F5F0E5F0F0
:106F200012560808E2F5F0E5F0125608245DF8E282
:106F3000785BE2547FF5F0785FE2C36001D3E5F05F
:106F400092E7F5F0E5F012560875F000E5F01256FC
:106F500008E53712560874FF1256083099FD12964C
:106F60005922C2B61214ABC0E07537007403125632
:106F700008E51E125608E51F125608744E125608F0
:106F800074041256087402125608740212560878D5
:106F9000B6E2F5F0E5F0125608D0F0E5F01256082A
:106FA000E53712560874FF1256083099FD129659AB
:106FB00022C0F088F0C0F0C2AF7882E2F54908E262
:106FC000F54AD2AFD0F0A8F0D0F0026FF9C0F08847
:106FD000F0C0F0C2AF7882E2F549F5F008E2F54A78
:106FE000D2AF45F0D0F0A8F0D0F0700DB21520155A
:106FF00008127007D24CD24722D21580F7C2AF7563
:1070000049FF754AFFD2AFC213C21522C217C2A0F0
:10701000028321D217D2A0028321304E14201511F1
:10702000543F4400C2AFF51A7519087518C002978D
:107030002322D2B3C294D2B4D2B2C32212749E50CD
:10704000F1C2B4D2B212964175F0FAC0F0D29412E5
:107050009671D0F020B2DBC0F0C2941296711296F5
:1070600071D0F030B2CCD5F0E2D2B3C294D2B4D267
:10707000B2D3222222227879B600FA75790274FFFF
:1070800002708B7879B600ED757901C0F0C0E074BC
:1070900010801075790274FF8003757901C0F0C00B
:1070A000E0741178A8760A0875F00A84F608A6F04C
:1070B000753B03D0E078BAF208D0E0F222C28C75BA
:1070C0008A45758C5DD28C30010C200209C0E0E548
:1070D000F914F5FED0E0B20020000132C0D0C0E0CB
:1070E000C0F075D008E581240B402F051DD2462045
:1070F00075171212C512721FE51D20E00C20E10960
:10710000301D1BE51D543F6077201D04E54860FEDF
:1071100012970DD0F0D0E0D0D032D26980EB204B66
:1071200005A215B392A2E51D30E22530E3031281DA
:10713000EA201D0312811AC3E562700EA217E56BE7
:1071400054406006E5717002B01892A0E57A704C68
:10715000E51D541F702DD247C25A78B5E2D5E0061E
:10716000D259D25A743CF2127ED2E4B54535B559A3
:1071700048B56249B5724AB5734BE51D543F70037B
:10718000B54746E4B5482EB5464DB5434EB54B52CE
:10719000B57657B577581271F2027109D57AB1D226
:1071A0007180ADD545C8C2137571007407127E6930
:1071B000D23CE480B9154880CE155980B415628060
:1071C000B3157280B2157380B1D547B775440530D9
:1071D0001D030264B380AC154680AFD543AFD240E7
:1071E00080ABD54BAB127B3A80A6157680A5157780
:1071F00080A4E54A45496026E54A2401F54A500243
:10720000054945497018C213204D13204E10301601
:1072100006E56D54407007127007D24CD24722E544
:107220001DA2E330480292A330490492A4D2A330B5
:107230004B0292A2304A0292A122C2B6204102D24F
:10724000B61272453212724DC2BCD2AC2275C80061
:10725000C2ADC2AC75CBFF75CA9885CBCD85CACC03
:10726000759853C298C29975C83475990622600CF6
:1072700014600914600D14601114601575F0FF742A
:1072800098801375F0FF74CC800C75F0FF74DE806D
:107290000575F0FF74E685F0CBF5CA75C834227524
:1072A000C800C2ACC2AD75980075CCC075CDE0D237
:1072B000AD75C8042275C800C2ACC2AD759800E5B2
:1072C0008A24C0F5CC540F658C24E0F5CDD2AD7581
:1072D000C80422C2A8C2AAC289C28BC2ACC2A9C2B7
:1072E000ABC2A3C248C2A2C24BC2A1C24AD2A4C26C
:1072F00049758F01D2A0120687D21D127013126F2A
:10730000FDE47887F27886F278A275F010F2D5F075
:10731000FCC24DC24EC24F753CFF753EFF751D0449
:10732000C2391296F37407127E95754700C23CD29B
:1073300046756500C21FC220D240C241754310E4A9
:10734000F53FF540F541F534F5361223AF751E30A3
:10735000751F30E4F545F54DF54CF550F551F53D0B
:10736000C222C223C22474557890F27891F27892A6
:10737000F27893F2D228754405754601C21A785006
:10738000E47A07F208DAFC754FFF787DA64FC21B3E
:10739000C21275720375591E755A00C254C213C2C7
:1073A00014C216C272C250C251755700755600758C
:1073B000F008785DE4F208D5F0FB7957E4F309F3BF
:1073C0007959F309F3785BE4F21218E47548FA127C
:1073D000970D7532FF7533FFD255756100785C7477
:1073E0000AF2756200C20EC20F756800756900125C
:1073F0006CFEE478BCF278BDF278BEF278BFF27829
:10740000B5743CF2C25DC25BC25CC25EC2187571EB
:1074100000127E52C25FD260C26178837600D2636E
:10742000757600757700C26DC26E754B00C270C272
:1074300071757A0078C17400F2789DE4F2C273C26B
:1074400075C274758901758A3E758C5DC2B9D2A901
:10745000D28CD2B6127245D2AFD2B4C294D2B31289
:10746000970DC269D26A22C2AF020000200F0A2023
:107470000E02C322127AD6D322127C47D32275F091
:1074800000C0F0128550D0F0500343F008C0F01255
:107490008562D0F0500343F010E5F022C322D2A061
:1074A00000000020A0F612964120A0F0D322758E95
:1074B00011758F0175A7079002FF7466F0E4E0B4C0
:1074C000665A9002FF7499F0E4E0B4994F759A6699
:1074D000E59AB46613759A99E59AB4990BD201D2DC
:1074E00002758F0175A7072275AC66E5ACB46624FA
:1074F00075AC99E5ACB4991CD201C20275D800757F
:10750000D94075F90075E90075DE0875EEFF75FE66
:10751000FFD2DE22C201D202758F0122C201C20255
:10752000221212C57548FA12970D12964112970D44
:1075300012964112970D22C2AF7581B575D00078B1
:10754000FF763E1274AE127521D2A01272D3126E63
:1075500065126D4512749E50030220E0126653506E
:10756000031267E812211E7548FA12252E500012E8
:107570000D0512746C754E031233E11233F71200CD
:10758000F0C2AF751880751903751A03129723D2CC
:107590001E30120C12162A120A57126D051217808D
:1075A000D2AFC21DC21E12749E50030220E0306989
:1075B0004DC2AF7518C0751900751A6312972380F4
:1075C0001EC2AF7518C0751900751A621297238014
:1075D0000EC2AF7518C0751900751A58129723D2CC
:1075E000B67581B5C26975F0FA129625D5F0FA75AF
:1075F000F0FA129625D5F0FA126D2F027467E58124
:10760000B4B5BE78FFB63EC930122E120A577401C7
:10761000105901E4C0E0120BD1D0E0120C34E57136
:1076200060021571301212121734126D86126DD766
:10763000126E83126D05126C53E55A6003D55A0B16
:10764000123532126C06126C40800CD2A3C248C2B2
:10765000A1D24AD2A4C249E5597003126D2FC24B80
:10766000D2A1C24A126E777896E2600D24FD4009DD
:1076700075670212362B12746C7897E2600D24FD48
:10768000400975670312362B12746CE56A5440602A
:107690000620A80312932FC250C251D24CD26E12B0
:1076A0002FF7C26E2043092042062044030276CE03
:1076B000302A0A7406127EB250030276C31246279D
:1076C00012746C785CE215E0F2600302761E785C5E
:1076D0007414F20275A00074A212776BE81277A6F8
:1076E000E91277A61277DD2274A212776BE812777F
:1076F000A6E71277A609D582F81277DD2274A212C6
:10770000776BE81277A674A312776B1277C6F70926
:10771000D582041277DD22C296D297000000C2976C
:1077200080E974A212776BE81277A612772F227481
:10773000A312776B1277C6F91277DD2274A27A084A
:10774000C296000000C297335005D296027751C20C
:1077500096D297000000C297DAEDD29600D2970039
:107760000000309604C297C322D3227A08D296D260
:107770009700000000000000000000000000000072
:1077800000C296000000C297335005D2960277924D
:10779000C296D297000000C297DAEDD29600D29737
:1077A000000000C297227A08335005D2960277B2C1
:1077B000C296D297000000C297DAEDD29600D29717
:1077C000000000C297227A08D296C29700000000FB
:1077D000D297C3309601B333DAF0C29722C2960033
:1077E0000000D297000000D2962278117994C082CE
:1077F0007582051276FDD0827894B6871408B6E0BB
:107800001008B6330C08B6A908789DE254FBF2C301
:1078100022789DE24404F2D3221277EA40012278D2
:107820008E76000876000876000876010876010852
:107830007600788C76000876007890E6543FF678EB
:1078400000798CC0827582071276E8D08212962564
:10785000C0E07993E7F9D0E078101276D712962538
:107860007815798CC0827582071276E8D0821296DC
:1078700025789476870876E00876330876A978111B
:107880007994C0827582041276E8D08212962578A7
:107890009DE254FBF2227802798EC0827582051235
:1078A00076FDD0827810127722E97993F77891E605
:1078B000232354037893665403601106C0E0799340
:1078C000E7F9D0E078101276D712962522788CE668
:1078D00075F018A4C0E07890E6C4540375F00AA4CB
:1078E000F5F0E6540F25F0D0F025F075F03CA4C07B
:1078F000F0C0E0788FE6C4540775F00AA4F5F0E60E
:10790000540F25F0D0F025F0F5F0D0E03400C5F0AC
:10791000221278967892E630E402240A540FFA781C
:1079200091E6C4540375F00AA4F5F0E6540F25F06F
:10793000FB7890E6C4540375F00AA4F5F0E6540F02
:1079400025F0FC788FE6C4540775F00AA4F5F0E63C
:10795000540F25F0FD7892E603C45407FE22122549
:107960000EC0D0127911D0D0501FBA0A12BE000F2B
:10797000EB24E7500ABC0202D322BC030280F98A3E
:10798000F0C0F01224F1D0F0FAC32212795E40293F
:10799000BE0026EB24E75021BA030CBC021B7890F2
:1079A00076031278328010BA0A0FBC030C789076F6
:1079B000021278321224EDD322C322788CA61E083C
:1079C000A61F08E51EF4F608E51FF4F67840798C4A
:1079D000C0827582041276E8D08212962522784001
:1079E000798CC0827582041276FDD082788CE6F4A0
:1079F000788E66700B788DE6F4788F667002C322FD
:107A0000D322C0E0791FE7F9D0E078401276D71290
:107A10009625C0E0791FE7F9D0E078411276D712B9
:107A20009625C0E0791FE7F9D0E078421276D712A8
:107A30009625C0E0791FE7F9D0E078431276D71297
:107A4000962522305F27205621C0D0C0E0E8C0E054
:107A5000C0F0E54B7003756300754B02C257127B93
:107A600004D0F0D0E0F8D0E0D0D0C289322056293E
:107A7000C0D0C0E0E8C0E0C0F0E54B70087563001E
:107A800078657400F2754B02A2B3B39257127D0869
:107A9000D0F0D0E0F8D0E0D0D0C28932C2AAC28BF8
:107AA00032305FF8205621C0D0C0E0E8C0E0C0F01E
:107AB000E54B7003756300754B02D257127B04D0FF
:107AC000F0D0E0F8D0E0D0D0C28B32C2A8C2AAC2B7
:107AD000B4C294129625D25FC2B4C294C289C28B3A
:107AE000D2B2D2B3C256754B00756300C2B8D28809
:107AF000D2A8C2BAD28AD2AA22C25FC2A8C2AAC2DD
:107B000089C28B22E56375F00884B41004756300A4
:107B10002250FA246FF8E2A25733F2056322E5639C
:107B200075F00884246FF8E5F0600E7408C395F0D2
:107B3000F5F0E2C333D5F0FBF222305F1D20561A78
:107B4000C0E0EFC0E0E56324F05007127B1ED25680
:107B50008003127AD6D0E0FFD0E022EF75F00884DF
:107B600005F0246FF8E233D5F0FC22E563C313C0BF
:107B7000E0500104C0E0C2577F00C0E0127B5BD040
:107B8000E05002B2570FD5E0F1D0E0D0F020571806
:107B9000C257AFF0C0E0127B5BD0E05002B2570F8B
:107BA000D5E0F1305702C322D32279657A0AE4F393
:107BB00009DAFCAF631F3057011F796E7A04127B1C
:107BC0005BE392E413F3DA0E540FF37A0419C3E97A
:107BD00094655002801FDFE620570C127B5BE39216
:107BE000E413F3DA08800BEA24FC6009E3C2E4132F
:107BF000DAFB540FF3E56330570224FEF56424D713
:107C0000500375642822127B6B4006D257127BAA60
:107C1000C322C257127BAAC322754632127ACB30D6
:107C20004605C246120273E54660083056F1127AE4
:107C3000F9C322127AF9D322C2A8C2AAC2B4C2944A
:107C4000C0E0129625D0E0C25FC2B4C294C289C21D
:107C50008BD2B2D2B3C256754B00756300C26BC2F1
:107C60006C757800C2B8D288D2A822754632127CD0
:107C700038304605C246120273E546600C3056F1B4
:107C8000E5637005127AD6C322127AD6D322C330A6
:107C9000E001B330E101B330E201B330E301B330CE
:107CA000E401B3227868E26017B409047408800222
:107CB00050FAF5F00879A8E2F70809D5F0F9C322DF
:107CC000D322E563B40F3BE220E439540FF5F018FA
:107CD000E230E430540F65F0702AE5F0B40B11E5A2
:107CE000787868F2D26CD256757800756300801788
:107CF000E57824EB400EE5782469F8E5F0F20578A4
:107D000080054003127C4722E56375F00584C0E0DE
:107D100024E7D0E040612465F8E2A25792E503F23F
:107D2000E5637014E2541FB40B07C26B75630580E2
:107D300045B40E42D26B80F40563206B85E5F0B448
:107D40000434E2127C8E502F540FF218E2540FB418
:107D50000F24D3E894657865F20404C082F5827537
:107D6000F00B08E265F0F5F0D582F7D082540F7081
:107D700006D25675630022127C47220100000000E3
:107D800000000000000A00000000000000000004E5
:107D9000060000000000000000080E0300000000C4
:107DA00000000000010702000000000000000A06B9
:107DB00008010000000000000402040F00000000A1
:107DC00000000806090809000000000000010E0577
:107DD0000F0500000000000A0C0A090B0300000058
:107DE00000040E0B00040502000000080E06070840
:107DF00004070100000001050A040D080E75F00AD1
:107E0000799C770009D5F0FA7865E2FA6042082497
:107E1000F25007EA24F328F87A0DE2540FF26028B2
:107E2000EA1475F00AA4247BF582E4347DF58379A5
:107E3000A57E007B0AE493F5F0E2A42E2775F010EE
:107E400084FEA7F0A319DBED08DACF756428C322FE
:107E5000D3229001FB75F008E4F0A3D5F0FB22C01B
:107E6000E0127EB2D0E0B3502CC0E024F8D0E04065
:107E700022C082C083F5F02403F582E43402F58346
:107E8000E0C5F024FBF582E43401F583E5F0F0D0A1
:107E900083D082D322C0E024F8D0E04013C082C057
:107EA0008324FBF582E43401F583E4F0D083D082AF
:107EB000C322C0E024F8D0E04016C082C08324FB77
:107EC000F582E43401F583E0D083D0826002D322CE
:107ED000C322C082C0839001FB75F008E06003B448
:107EE000FF09A3D5F0F6D083D0822220E70414F056
:107EF00080F0305AED14F0B480E8E4F080E4B4404F
:107F0000087400127EB2027FADB441087401127E83
:107F1000B2027FADB442087402127EB2027FADB4E9
:107F200043087403127EB2027FADB4440774041296
:107F30007EB28079B45407A2677268B3806FB4557B
:107F400006A267B0688066B45606A268B067805D16
:107F5000B45706A26782688054B45807A265726657
:107F6000B3804AB45906A265B0668041B45A06A2ED
:107F700066B0658038B45B06A2658266802FB46106
:107F800007301428A2158025B4620720141EA215FC
:107F9000801BB46304A2158014C0E024D9D0E04053
:107FA00012232422C0E0E43480C0E022C374012202
:107FB000D380FAE4C322A238B380F2D247A2188059
:107FC000EC80F0A21380E6A21680E2A26180DE803F
:107FD000DF80E0A21480D6E56260D180D3E56845F9
:107FE0006960C980CB126A4F80C3A24F724EB380C2
:107FF000BCA24E821580B6A24EB01580B0A24F80B2
:10800000ACC3305D0920380678BEE27001D3809D94
:10801000A217509CE56B54406092E571708EA218D7
:10802000808B8092809580938091808F808D808BD3
:108030008089808D808D808F8091809380938093C4
:1080400080958099809F80A280A780AB80AF80B10F
:1080500080BE802E8035803F8049804C804D804E90
:10806000804F8057805C806180068009800C800E84
:10807000A238027FADA272027FADC3027FADC30200
:108080007FADC3E5726001D3027FADC3203805E543
:10809000736001D3027FADC3303805E5736001D34F
:1080A000027FADA263027FAD0280E70280F8028109
:1080B00009E5766003027FB0027FACE57760F902E4
:1080C0007FB0A273725C027FADA273725C5010E548
:1080D0001D54F8B48004D3027FADB4900280F7C37E
:1080E000027FADC3027FADE56B541060033038F3FF
:1080F0007405127EB2027FADE56B54106003303818
:10810000E27406127EB2027FADE56B54106003305C
:1081100038D17407127EB2027FAD301219C0E0C0B0
:1081200082C0837403120189D083D082D0E04003DF
:10813000028151028136E538B4FF027463B40D0A3E
:10814000300902801ED209D38015127EFE60148091
:108150000EE538B40D06200903028163C209C392FB
:1081600006D26A301219C0E0C082C08374041201C2
:1081700089D083D082D0E0400302819502817FE5DF
:1081800039B40D0A300A02801ED20AD38015127E3D
:10819000FE6014800EE539B40D06200A030281A7A3
:1081A000C20AC39207D26A301219C0E0C082C083EB
:1081B0007405120189D083D082D0E040030281D9B6
:1081C0000281C3E53AB40D0A300B02801CD20BD3F6
:1081D0008015127EFE6012800EE53AB40D06200B6B
:1081E000030281E9C20BC3920822E56B54106003BD
:1081F000303827E56C540470077405127EB2404095
:10820000E56C540170077406127EB24015E56C549B
:108210000270077407127EB24017C218754D000233
:108220008256E54DB401028024754D01754C4080A5
:108230001CE54DB402028015754D02754CA0800DF1
:10824000E54DB403028006754D03754CF0E54C23F3
:10825000F54CA2E0921822C207D26A22D207D26A53
:1082600022B207D26A22F5F00303543FB40258E564
:108270003964086005E539B40D4AE5F089F0C0F0CD
:10828000301219C0E0C082C0837404120189D08307
:10829000D082D0E040030282AB02829CD0F0A9F0F1
:1082A0005403B4020D12825702831FD0F0A9F002CA
:1082B000831FB4010612825C02831FB4030612827C
:1082C0006102831F02831DB40353E53A640860050D
:1082D000E53AB40DEFE5F089F0C0F0301219C0E0D6
:1082E000C082C0837405120189D083D082D0E0405F
:1082F000030283050282F7D0F0A9F05403B4020C04
:10830000C20802831FD0F0A9F002831FB40105D276
:108310000802831FB40304B20880048000D322C380
:1083200022C0E07417301716B53804C206D26AB5F9
:108330003904C207D26AB53A02C208D0E022B53881
:1083400004D206D26AB53904D207D26AB53A02D24B
:1083500008D0E022C0E0128542D0E0402530290359
:1083600020381F204F1CC0E012701AC214126FCDAB
:10837000D0E020320BC2AF1295CE751810129723A1
:10838000D32220320BC2AF1295CE7518201297233C
:10839000C322D216757610C2AF7518C07519007554
:1083A0001A01129723301526204E2E20300DC2AF11
:1083B0007549FF754AF8D2AF1270077884E2F54527
:1083C000E56D5410600312553E787F76FF22788465
:1083D000E2F545202E0312848122C24FC24E204D69
:1083E00009C0E0126FFDD0E0D24C543F44C0C2AF90
:1083F000F51A7519087518C0029723D24FC24E207E
:108400004D09C0E0126FFDD0E0D24C543F4480C211
:10841000AFF51A7519087518C0029723D24EC24FCE
:10842000204D09C0E0126FFDD0E0D24C543F4440D3
:10843000C2AFF51A7519087518C0029723D24EC23B
:108440004F204D09C0E0126FB1D0E0D24C543F44F0
:1084500000C2AFF51A7519087518C0029723E56DAB
:108460005440600312700722C2167545007407124B
:108470007E95C2AF7518C0751900751A0212972340
:10848000227571007405127E69C2AF751850751996
:108490000F751AFF12972322C238D263C2AF751824
:1084A0006075190F751AFF1297231255A375730380
:1084B000120C7A1296FDC23A22D238C263C2AF754C
:1084C000187075190F751AFF12972312559475734A
:1084D00003120C7A22C0E0C082C0831267E8D08306
:1084E000D082D0E0543F4400C2AFF51A75190B7525
:1084F00018C012972322789EF208F208F208F2C000
:10850000E01234A0D0E07010C2AF7518C075190029
:10851000751A50129723C322C2AF7518C07519007F
:10852000751A5C129723C322400C304D08C24D20AF
:108530004E03126FFD22204DFC12701A126FB1D241
:108540004D221289274008128D9240031291FD227C
:10855000C320380D1289324008128D9D40031292BB
:108560000822203814E56E5480600E12893D40F1D7
:10857000128DA840EC12921322C322A203302501CF
:10858000B37890E233F2221060030289E5301D08CF
:10859000C37890E4F2028948E56C541060033038E7
:1085A000EF7890E260EF0460030289E3788CE2B434
:1085B0000302800620280320224FD222301219C045
:1085C000E0C082C0837400120189D083D082D0E0E1
:1085D00040030289E30285D8788CE224A4401CC0C1
:1085E00082C08390886FE225E00493F5F0E225E0F5
:1085F00093D083D082C0F0C0E0E222E2C2AF75180F
:1086000090751909F51A1297230289E3126E7712F1
:1086100000D60289E374011283920289E37401C2D5
:108620001412835440030289E302860CD31293FD93
:108630000289E37562050285FCC0E07401127E695F
:10864000D0E00285FC203803202F0CC0E074041217
:108650007E69D0E00285FC0289E3743D02875C02FA
:1086600085FCD24CC0E0E56D54047005D0E0028575
:10867000FCD0E00289E3C0E0D37401128528D0E089
:108680000285FC7401D21412835440030289E30270
:10869000860C75F0051270760289E375F00512708C
:1086A000930289E30285FC0285FCE475F0051270F3
:1086B000830289E3741075F0051270830289E374F4
:1086C0001175F0051270830289E3742075F00512AC
:1086D00070830289E37401F9748CF8752F0075308A
:1086E0008C7531F1120539788CE675F005127083BE
:1086F0000289E37401F9748CF8752F0075308C755C
:1087000031F1120539788CE675F00512709A0289FC
:10871000E312128160167401543F4480C2AF751891
:10872000C0751909F51A12972302860C0289E330E5
:108730005D1AE478BEF27401543F4440C2AF75182C
:10874000C0751909F51A12972302860C12129D5052
:10875000DB02873674011284D502860C203813128E
:108760008550401A12856240151284B9757A1F022D
:10877000860C128498757A1F1212AF02860C028939
:10878000E3E56A54106007E41284F602860C02895D
:10879000E3E56A5410600874FF1284F602860C0246
:1087A00089E374011283DA0289E3740112843D02C1
:1087B00089E3740112841C0289E374011283FB02B1
:1087C00089E37400127E69740112968D02860C741E
:1087D00000127E95740112969E02860C7400127E21
:1087E000B240EC0287C27402127E6974011296AF25
:1087F00002860C7402127E9574011296C002860CD9
:108800007402127EB240EC0287E67403127E697431
:10881000011296D102860C7403127E957401129691
:10882000E202860C7403127EB240EC02880A3038F1
:10883000030287720289E32038FA02875F740044DA
:10884000011293E702860C744002883F748002880C
:108850003F74C002883F740044011293D102860C19
:108860007440028858748002885874C002885889FD
:10887000E38615861D862C85FC85FC85FC86338663
:10888000398645865A85FC865F8662867685FC85B4
:10889000FC85FC85FC85FC85FC85FC85FC85FC85D0
:1088A000FC85FC85FC85FC85FC85FC85FC85FC85C0
:1088B000FC85FC85FC85FC85FC85FC85FC85FC85B0
:1088C000FC85FC85FC85FC85FC85FC85FC86838617
:1088D00092869B86A486A786AA86B486BF86CA8609
:1088E000D586F38711872F8754875C878187918787
:1088F000A287AA87B287BA87C287CF87DC87E68735
:10890000F38800880A8817882485FC882E88378594
:10891000FC85FC85FC85FC883D8847884C8851880F
:108920005688608865886A788CE2B40B03A222229C
:10893000C322788CE2B40D03A22222C322788CE2F7
:10894000B40103A22222C322788CE2B4030280097C
:108950002028062022030289E3C222301219C0E037
:10896000C082C0837400120189D083D082D0E040DD
:10897000030289E3028977788CE260DAB401091294
:10898000845E1284680289E3B402030289E3B403BB
:108990000B128550404DC31293FD8047B409082047
:1089A0003832302F2F803CB40A02743DB40D0DD202
:1089B0004CE56D5404702C740D0289D4B40E0BC3B5
:1089C0007401128528740E0289D4B41E004005B4C7
:1089D0006400400FC2AF7518A0751909F51A1297F7
:1089E000238000D26022A204302601B37891E233C2
:1089F000F222106003028E50301D08C37891E4F219
:108A0000028DB3E56C542060033038EF7891E2605A
:108A1000EF046003028E4E788DE2B40302800620DC
:108A2000280320234FD223301219C0E0C082C08314
:108A30007401120189D083D082D0E04003028E4EAF
:108A4000028A43788DE224A4401CC082C083908CAB
:108A5000DAE225E00493F5F0E225E093D083D082BA
:108A6000C0F0C0E0E222E2C2AF75189075190AF5B5
:108A70001A129723028E4E126E771200D6028E4E75
:108A80007402128392028E4E7402C21412835440F6
:108A900003028E4E028A77D31293FD028E4E7562C8
:108AA00005028A67C0E07401127E69D0E0028A671D
:108AB000203803202F0CC0E07404127E69D0E0023D
:108AC0008A67028E4E743D028BC7028A67D24CC001
:108AD000E0E56D54047005D0E0028A67D0E0028EB4
:108AE0004EC0E0D37402128528D0E0028A67740277
:108AF000D2141283544003028E4E028A7775F00519
:108B0000127076028E4E75F005127093028E4E0230
:108B10008A67028A67E475F005127083028E4E74CC
:108B20001075F005127083028E4E741175F00512E7
:108B30007083028E4E742075F005127083028E4E83
:108B40007401F9748CF8752F0075308C7531F5123D
:108B50000539788CE675F005127083028E4E74012B
:108B6000F9748CF8752F0075308C7531F512053954
:108B7000788CE675F00512709A028E4E12128160A2
:108B8000167402543F4480C2AF7518C0751909F5B8
:108B90001A129723028A77028E4E305D1AE478BE4D
:108BA000F27402543F4440C2AF7518C0751909F5FC
:108BB0001A129723028A7712129D50DB028BA1743E
:108BC000021284D5028A77203813128550401A1277
:108BD000856240151284B9757A1F028A77128498CB
:108BE000757A1F1212AF028A77028E4EE56A541010
:108BF0006007E41284F6028A77028E4EE56A54100A
:108C0000600874FF1284F6028A77028E4E74021294
:108C100083DA028E4E740212843D028E4E7402126A
:108C2000841C028E4E74021283FB028E4E7400125C
:108C30007E69740212968D028A777400127E957492
:108C40000212969E028A777400127EB240EC028C69
:108C50002D7402127E6974021296AF028A77740232
:108C6000127E9574021296C0028A777402127EB246
:108C700040EC028C517403127E6974021296D10288
:108C80008A777403127E9574021296E2028A7774D0
:108C900003127EB240EC028C75303803028BDD0289
:108CA0008E4E2038FA028BCA740044021293E702F7
:108CB0008A777440028CAA7480028CAA74C0028CD9
:108CC000AA740044021293D1028A777440028CC3C2
:108CD0007480028CC374C0028CC38E4E8A808A88D2
:108CE0008A978A678A678A678A9E8AA48AB08AC5B1
:108CF0008A678ACA8ACD8AE18A678A678A678A67A9
:108D00008A678A678A678A678A678A678A678A67DB
:108D10008A678A678A678A678A678A678A678A67CB
:108D20008A678A678A678A678A678A678A678A67BB
:108D30008A678A678A678A678AEE8AFD8B068B0F45
:108D40008B128B158B1F8B2A8B358B408B5E8B7C0C
:108D50008B9A8BBF8BC78BEC8BFC8C0D8C158C1D71
:108D60008C258C2D8C3A8C478C518C5E8C6B8C7541
:108D70008C828C8F8A678C998CA28A678A678A67B3
:108D80008A678CA88CB28CB78CBC8CC18CCB8CD0F5
:108D90008CD5788DE2B40B03A22322C322788DE216
:108DA000B40D03A22322C322788DE2B40103A223CF
:108DB00022C322788DE2B4030280092028062023F2
:108DC00003028E4EC223301219C0E0C082C08374E9
:108DD00001120189D083D082D0E04003028E4E027E
:108DE0008DE2788DE260DAB4010912845E12846843
:108DF000028E4EB40203028E4EB4030B1285504015
:108E00004DC31293FD8047B40908203832302F2F0C
:108E1000803CB40A02743DB40D0DD24CE56D54048F
:108E2000702C740D028E3FB40E0BC3740212852891
:108E3000740E028E3FB41E004005B46400400FC2A1
:108E4000AF7518A075190AF51A1297238000D26021
:108E500022A205302701B37892E233F22210600398
:108E60000292BB301D08C37892E4F202921EE56CB8
:108E7000544060033038EF7892E260EF0460030200
:108E800092B9788EE2B40302800620280320244F92
:108E9000D224301219C0E0C082C08374021201894A
:108EA000D083D082D0E040030292B9028EAE788E99
:108EB000E224A4401CC082C083909145E225E004D6
:108EC00093F5F0E225E093D083D082C0F0C0E0E2D9
:108ED00022E2C2AF75189075190CF51A1297230289
:108EE00092B9126E771200D60292B974031283926D
:108EF0000292B97403C21412835440030292B9025D
:108F00008EE2D31293FD0292B9756205028ED2C031
:108F1000E07401127E69D0E0028ED2203803202F47
:108F20000CC0E07404127E69D0E0028ED20292B9C5
:108F3000743D029032028ED2D24CC0E0E56D5404F2
:108F40007005D0E0028ED2D0E00292B9C0E0D374B6
:108F500003128528D0E0028ED27403D214128354F7
:108F600040030292B9028EE275F005127076029209
:108F7000B975F0051270930292B9028ED2028ED2A8
:108F8000E475F0051270830292B9741075F0051241
:108F900070830292B9741175F0051270830292B950
:108FA000742075F0051270830292B97401F9748C03
:108FB000F8752F0075308C7531F7120539788CE60D
:108FC00075F0051270830292B97401F9748CF8750A
:108FD0002F0075308C7531F7120539788CE675F0F5
:108FE0000512709A0292B912128160167403543FEE
:108FF0004480C2AF7518C0751909F51A129723027B
:109000008EE20292B9305D1AE478BEF27403543FE6
:109010004440C2AF7518C0751909F51A129723029A
:109020008EE212129D50DB02900C74031284D50262
:109030008EE2203813128550401A128562401512B4
:1090400084B9757A1F028EE2128498757A1F121203
:10905000AF028EE20292B9E56A54106007E412840E
:10906000F6028EE20292B9E56A5410600874FF12AB
:1090700084F6028EE20292B974031283DA0292B984
:10908000740312843D0292B9740312841C0292B9D3
:1090900074031283FB0292B97400127E6974031286
:1090A000968D028EE27400127E95740312969E02D3
:1090B0008EE27400127EB240EC0290987402127E2E
:1090C0006974031296AF028EE27402127E957403E5
:1090D0001296C0028EE27402127EB240EC0290BC84
:1090E0007403127E6974031296D1028EE274031225
:1090F0007E9574031296E2028EE27403127EB240F1
:10910000EC0290E03038030290480292B92038FA1D
:10911000029035740044031293E7028EE274400219
:109120009115748002911574C00291157400440366
:109130001293D1028EE2744002912E748002912E1D
:1091400074C002912E92B98EEB8EF38F028ED28E66
:10915000D28ED28F098F0F8F1B8F308ED28F358F8B
:10916000388F4C8ED28ED28ED28ED28ED28ED28E1E
:10917000D28ED28ED28ED28ED28ED28ED28ED28EEF
:10918000D28ED28ED28ED28ED28ED28ED28ED28EDF
:10919000D28ED28ED28ED28ED28ED28ED28ED28ECF
:1091A000D28ED28F598F688F718F7A8F7D8F808FFB
:1091B0008A8F958FA08FAB8FC98FE79005902A90EB
:1091C0003290579067907890809088909090989087
:1091D000A590B290BC90C990D690E090ED90FA8E98
:1091E000D29104910D8ED28ED28ED28ED2911391C5
:1091F0001D91229127912C9136913B9140788EE2DE
:10920000B40B03A22422C322788EE2B40D03A2245D
:1092100022C322788EE2B40103A22422C322788ED4
:10922000E2B4030280092028062024030292B9C276
:1092300024301219C0E0C082C0837402120189D0A8
:1092400083D082D0E040030292B902924D788EE240
:1092500060DAB4010912845E1284680292B9B40221
:10926000030292B9B4030B128550404DC31293FD13
:109270008047B40908203832302F2F803CB40A02CE
:10928000743DB40D0DD24CE56D5404702C740D0278
:1092900092AAB40E0BC37403128528740E0292AA0C
:1092A000B41E004005B46400400FC2AF7518A0752D
:1092B000190CF51A1297238000D2602212137EE552
:1092C0006A5440601AE56B5402700612857B128561
:1092D00087E56B540470061289E61289F2800C123D
:1092E000857B1285871289E61289F2128E51128EC1
:1092F0005DC228203C0122C23CC2AF7518C075195E
:1093000000751A5412972322E8C0E0788CE26403B7
:109310006018788DE264036011788EE26403600A5D
:10932000788FE264036003C38001D3D0E0F822E4C5
:10933000A20692E0A20792E1A20892E2F5667567A2
:109340000512341074035004123604221235DC78EE
:1093500085E6C0E0E56B54026012D0E0C0E054073F
:10936000129389D0E0C0E05407129389E56B54044E
:109370006014D0E0C0E0C454071293ADD0E0C0E068
:10938000C454071293ADD0E022A222302501B3408D
:1093900007D320E10A0293ACC320E2030293AC306E
:1093A0002501B3E494007890F212858722A223303D
:1093B0002601B34007D320E10A0293D0C320E20381
:1093C0000293D0302601B3E494007891F21289F22E
:1093D00022A2E69265A2E79266C2AFF51A75190D50
:1093E0007518C012972322A2E69267A2E79268C27C
:1093F000AFF51A75190F7518C012972322C0D0E562
:109400007A600302942B307105C2711200AAD0D089
:10941000203801B350142038091284B9126E77D263
:109420004C22128498126E77D24C22D0D020380170
:10943000B340F7757A00126E7722E9C4540F2323E4
:10944000F890958E93FF08E893FE08E893FD08E8EE
:1094500093FCE9540F601BF82328F890955E932F36
:10946000D4FF08E8933ED4FE08E8933DD4FDE43CE5
:10947000D4FCEA603CC4540F601BF82328F8909594
:1094800031932FD4FF08E8933ED4FE08E8933DD4EF
:10949000FDE43CD4FCEA540F601723F89095149334
:1094A0002FD4FF08E8933ED4FEE43DD4FDE43CD441
:1094B000FCEB6034C4540F601723F89094F6932F9C
:1094C000D4FF08E8933ED4FEE43DD4FDE43CD4FC54
:1094D000EB540F60139094E8932FD4FFE43ED4FE36
:1094E000E43DD4FDE43CD4FC22010203040506075C
:1094F00008091011121314151600320048006400F8
:109500008000960012012801440160017601920159
:109510000802240240025602120568072410801235
:1095200036159217482004236025162872302833F8
:10953000843540389640009281008822018463017E
:10954000800402764502728602682703646803601D
:1095500009045650045291044832054473054014DE
:109560000636550672101308661944212680763295
:10957000163239528745884252249858605365966E
:10958000087232647868198504759140309800003B
:109590000000768504015271090228571403044320
:1095A0001904802824055614290632003407088639
:1095B0003808847143096057481036435311122903
:1095C0005812881463136400681440867215B4013D
:1095D0000775190F751AE122B4020775190F751A6C
:1095E000E222B4030775190F751AE322B404077554
:1095F000190F751AE422B4110775190F751AD122C3
:10960000B4120775190F751AD222B4130775190F02
:10961000751AD322B4140775190F751AD422751947
:109620000F751AD422D2AFD28CC28E53890F4389C0
:1096300010758BD6758D97C28FD28E308FFDC28EEE
:1096400022C28E53890F438910758BEB758DCBC267
:109650008FD28E308FFDC28E22C28E53890F4389E6
:1096600010758B96758DF5C28FD28E308FFDC28EA0
:1096700022C28E53890F438910E58AC424C0F58B1A
:10968000758DE0C28FD28E308FFDC28E22543F4442
:1096900000C2AFF51A75190A7518C0029723543F16
:1096A0004480C2AFF51A75190A7518C00297235481
:1096B0003F4400C2AFF51A75190C7518C002972304
:1096C000543F4440C2AFF51A75190C7518C0029783
:1096D00023543F4480C2AFF51A75190C7518C002A7
:1096E0009723543F44C0C2AFF51A75190C7518C0C2
:1096F0000297237401127E957404127E95740712EA
:109700007E957406127E957405127E9522B2842091
:10971000010122200206E5F914F5FE2275A61E7548
:10972000A6E1223001030297AF53510F53500F535C
:1097300018F053190FC2AFE550232430F8E518454F
:1097400019F208E51AF2055053500FE550B55105CE
:10975000055153510FD2AFC3E5509551500224101B
:10976000C0E024F3D0E05002D27024F450037559C5
:109770000022300103029808E551B55004E4780056
:1097800022C3332430F8E2C0E008E2F8D0E022300F
:10979000010302982C53500F53510FC2AFE551B53E
:1097A0005004D2AFD322055153510FD2AFC322532D
:1097B000513F53503F5318F053190FC082C083C21A
:1097C000AFE55023240BF58275830250020583E533
:1097D000184519F0A3E51AF0D083D08205505350F4
:1097E0003FE550B55105055153513FD2AFC3E55048
:1097F000955150022440C0E024C4D0E05002D27001
:1098000024D0500375590022E551B55004E4780086
:1098100022C333C082C083240BF5827583025002B9
:109820000583E0F8A3E0C8D083D0822253503F5391
:10983000513FC2AFE551B55004D2AFD322055153C9
:10984000513FD2AFC3220000000000000000000022
:109850000000000000000000000000000000000008
:1098600000000000000000000000000000000000F8
:1098700000000000000000000000000000000000E8
:1098800000000000000000000000000000000000D8
:109BA0003C434647544147533E3C5645523D4D3158
:109BB0003534303E3C46495849443D20203E3C4ED9
:109BC000414D453D505233303276322E30332E31B6
:109BD0003534303E3C444154413D32352D30312DF9
:109BE00031302030323A30313E3C2F4346475441E9
:109BF00047533E000000000000000000000000F09D
:00000001FF
:0300000306028072
